BL51 BANKED LINKER/LOCATER V6.02                                                        04/19/2018  15:18:09  PAGE 1


BL51 BANKED LINKER/LOCATER V6.02, INVOKED BY:
C:\KEIL\C51\BIN\BL51.EXE fw.obj, dscr.obj, .\EZUSB.LIB, .\USBJmpTb.OBJ, interrupciones.obj, pedalera.obj, I2C.obj TO Int
>> erfazPedalera RAMSIZE (256) CODE (0X80-0X1FFF) XDATA (0X2000)


MEMORY MODEL: SMALL


INPUT MODULES INCLUDED:
  fw.obj (FW)
  dscr.obj (DSCR)
  .\EZUSB.LIB (RESUME)
  .\EZUSB.LIB (DISCON)
  .\EZUSB.LIB (EZREGS)
  .\EZUSB.LIB (GET_STRD)
  .\EZUSB.LIB (SUSP)
  .\EZUSB.LIB (DELAY)
  .\EZUSB.LIB (DELAY1MS)
  .\USBJmpTb.OBJ (USBJMPTBL)
  interrupciones.obj (INTERRUPCIONES)
  pedalera.obj (PEDALERA)
  I2C.obj (I2C)
  C:\KEIL\C51\LIB\C51S.LIB (?C_STARTUP)
  C:\KEIL\C51\LIB\C51S.LIB (?C?ULCMP)
  C:\KEIL\C51\LIB\C51S.LIB (?C?CCASE)
  C:\KEIL\C51\LIB\C51S.LIB (?C_INIT)


LINK MAP OF MODULE:  InterfazPedalera (FW)


            TYPE    BASE      LENGTH    RELOCATION   SEGMENT NAME
            -----------------------------------------------------

            * * * * * * *   D A T A   M E M O R Y   * * * * * * *
            REG     0000H     0008H     ABSOLUTE     "REG BANK 0"
            DATA    0008H     0015H     UNIT         _DATA_GROUP_
                    001DH     0003H                  *** GAP ***
            BIT     0020H.0   0000H.4   UNIT         ?BI?FW
            BIT     0020H.4   0000H.1   UNIT         ?BI?PEDALERA
            BIT     0020H.5   0000H.1   UNIT         _BIT_GROUP_
                    0020H.6   0000H.2                *** GAP ***
            DATA    0021H     001EH     UNIT         ?DT?PEDALERA
            DATA    003FH     000EH     UNIT         ?DT?FW
            IDATA   004DH     0001H     UNIT         ?STACK

            * * * * * * *  X D A T A   M E M O R Y  * * * * * * *
                    0000H     2000H                  *** GAP ***
            XDATA   2000H     0002H     UNIT         _XDATA_GROUP_
                    2002H     C3FEH                  *** GAP ***
            XDATA   E400H     0001H     ABSOLUTE     
                    E401H     007FH                  *** GAP ***
            XDATA   E480H     0001H     ABSOLUTE     
                    E481H     008CH                  *** GAP ***
            XDATA   E50DH     0001H     ABSOLUTE     
                    E50EH     00F2H                  *** GAP ***
            XDATA   E600H     0001H     ABSOLUTE     
            XDATA   E601H     0001H     ABSOLUTE     
BL51 BANKED LINKER/LOCATER V6.02                                                      04/19/2018  15:18:09  PAGE 2


            XDATA   E602H     0001H     ABSOLUTE     
            XDATA   E603H     0001H     ABSOLUTE     
            XDATA   E604H     0001H     ABSOLUTE     
            XDATA   E605H     0001H     ABSOLUTE     
            XDATA   E606H     0001H     ABSOLUTE     
            XDATA   E607H     0001H     ABSOLUTE     
            XDATA   E608H     0001H     ABSOLUTE     
            XDATA   E609H     0001H     ABSOLUTE     
            XDATA   E60AH     0001H     ABSOLUTE     
            XDATA   E60BH     0001H     ABSOLUTE     
            XDATA   E60CH     0001H     ABSOLUTE     
                    E60DH     0003H                  *** GAP ***
            XDATA   E610H     0001H     ABSOLUTE     
            XDATA   E611H     0001H     ABSOLUTE     
            XDATA   E612H     0001H     ABSOLUTE     
            XDATA   E613H     0001H     ABSOLUTE     
            XDATA   E614H     0001H     ABSOLUTE     
            XDATA   E615H     0001H     ABSOLUTE     
                    E616H     0002H                  *** GAP ***
            XDATA   E618H     0001H     ABSOLUTE     
            XDATA   E619H     0001H     ABSOLUTE     
            XDATA   E61AH     0001H     ABSOLUTE     
            XDATA   E61BH     0001H     ABSOLUTE     
                    E61CH     0004H                  *** GAP ***
            XDATA   E620H     0001H     ABSOLUTE     
            XDATA   E621H     0001H     ABSOLUTE     
            XDATA   E622H     0001H     ABSOLUTE     
            XDATA   E623H     0001H     ABSOLUTE     
            XDATA   E624H     0001H     ABSOLUTE     
            XDATA   E625H     0001H     ABSOLUTE     
            XDATA   E626H     0001H     ABSOLUTE     
            XDATA   E627H     0001H     ABSOLUTE     
            XDATA   E628H     0001H     ABSOLUTE     
            XDATA   E629H     0001H     ABSOLUTE     
            XDATA   E62AH     0001H     ABSOLUTE     
            XDATA   E62BH     0001H     ABSOLUTE     
            XDATA   E62CH     0001H     ABSOLUTE     
            XDATA   E62DH     0001H     ABSOLUTE     
            XDATA   E62EH     0001H     ABSOLUTE     
            XDATA   E62FH     0001H     ABSOLUTE     
            XDATA   E630H     0001H     ABSOLUTE     
            XDATA   E631H     0001H     ABSOLUTE     
            XDATA   E632H     0001H     ABSOLUTE     
            XDATA   E633H     0001H     ABSOLUTE     
            XDATA   E634H     0001H     ABSOLUTE     
            XDATA   E635H     0001H     ABSOLUTE     
            XDATA   E636H     0001H     ABSOLUTE     
            XDATA   E637H     0001H     ABSOLUTE     
                    E638H     0008H                  *** GAP ***
            XDATA   E640H     0001H     ABSOLUTE     
            XDATA   E641H     0001H     ABSOLUTE     
            XDATA   E642H     0001H     ABSOLUTE     
            XDATA   E643H     0001H     ABSOLUTE     
                    E644H     0004H                  *** GAP ***
            XDATA   E648H     0001H     ABSOLUTE     
            XDATA   E649H     0001H     ABSOLUTE     
                    E64AH     0006H                  *** GAP ***
BL51 BANKED LINKER/LOCATER V6.02                                                      04/19/2018  15:18:09  PAGE 3


            XDATA   E650H     0001H     ABSOLUTE     
            XDATA   E651H     0001H     ABSOLUTE     
            XDATA   E652H     0001H     ABSOLUTE     
            XDATA   E653H     0001H     ABSOLUTE     
            XDATA   E654H     0001H     ABSOLUTE     
            XDATA   E655H     0001H     ABSOLUTE     
            XDATA   E656H     0001H     ABSOLUTE     
            XDATA   E657H     0001H     ABSOLUTE     
            XDATA   E658H     0001H     ABSOLUTE     
            XDATA   E659H     0001H     ABSOLUTE     
            XDATA   E65AH     0001H     ABSOLUTE     
            XDATA   E65BH     0001H     ABSOLUTE     
            XDATA   E65CH     0001H     ABSOLUTE     
            XDATA   E65DH     0001H     ABSOLUTE     
            XDATA   E65EH     0001H     ABSOLUTE     
            XDATA   E65FH     0001H     ABSOLUTE     
            XDATA   E660H     0001H     ABSOLUTE     
            XDATA   E661H     0001H     ABSOLUTE     
            XDATA   E662H     0001H     ABSOLUTE     
            XDATA   E663H     0001H     ABSOLUTE     
            XDATA   E664H     0001H     ABSOLUTE     
            XDATA   E665H     0001H     ABSOLUTE     
            XDATA   E666H     0001H     ABSOLUTE     
            XDATA   E667H     0001H     ABSOLUTE     
            XDATA   E668H     0001H     ABSOLUTE     
                    E669H     0007H                  *** GAP ***
            XDATA   E670H     0001H     ABSOLUTE     
            XDATA   E671H     0001H     ABSOLUTE     
            XDATA   E672H     0001H     ABSOLUTE     
                    E673H     0005H                  *** GAP ***
            XDATA   E678H     0001H     ABSOLUTE     
            XDATA   E679H     0001H     ABSOLUTE     
            XDATA   E67AH     0001H     ABSOLUTE     
            XDATA   E67BH     0001H     ABSOLUTE     
            XDATA   E67CH     0001H     ABSOLUTE     
            XDATA   E67DH     0001H     ABSOLUTE     
            XDATA   E67EH     0001H     ABSOLUTE     
            XDATA   E67FH     0001H     ABSOLUTE     
            XDATA   E680H     0001H     ABSOLUTE     
            XDATA   E681H     0001H     ABSOLUTE     
            XDATA   E682H     0001H     ABSOLUTE     
            XDATA   E683H     0001H     ABSOLUTE     
            XDATA   E684H     0001H     ABSOLUTE     
            XDATA   E685H     0001H     ABSOLUTE     
            XDATA   E686H     0001H     ABSOLUTE     
            XDATA   E687H     0001H     ABSOLUTE     
                    E688H     0002H                  *** GAP ***
            XDATA   E68AH     0001H     ABSOLUTE     
            XDATA   E68BH     0001H     ABSOLUTE     
                    E68CH     0001H                  *** GAP ***
            XDATA   E68DH     0001H     ABSOLUTE     
                    E68EH     0001H                  *** GAP ***
            XDATA   E68FH     0001H     ABSOLUTE     
            XDATA   E690H     0001H     ABSOLUTE     
            XDATA   E691H     0001H     ABSOLUTE     
                    E692H     0002H                  *** GAP ***
            XDATA   E694H     0001H     ABSOLUTE     
BL51 BANKED LINKER/LOCATER V6.02                                                      04/19/2018  15:18:09  PAGE 4


            XDATA   E695H     0001H     ABSOLUTE     
                    E696H     0002H                  *** GAP ***
            XDATA   E698H     0001H     ABSOLUTE     
            XDATA   E699H     0001H     ABSOLUTE     
                    E69AH     0002H                  *** GAP ***
            XDATA   E69CH     0001H     ABSOLUTE     
            XDATA   E69DH     0001H     ABSOLUTE     
                    E69EH     0002H                  *** GAP ***
            XDATA   E6A0H     0001H     ABSOLUTE     
            XDATA   E6A1H     0001H     ABSOLUTE     
            XDATA   E6A2H     0001H     ABSOLUTE     
            XDATA   E6A3H     0001H     ABSOLUTE     
            XDATA   E6A4H     0001H     ABSOLUTE     
            XDATA   E6A5H     0001H     ABSOLUTE     
            XDATA   E6A6H     0001H     ABSOLUTE     
            XDATA   E6A7H     0001H     ABSOLUTE     
            XDATA   E6A8H     0001H     ABSOLUTE     
            XDATA   E6A9H     0001H     ABSOLUTE     
            XDATA   E6AAH     0001H     ABSOLUTE     
            XDATA   E6ABH     0001H     ABSOLUTE     
            XDATA   E6ACH     0001H     ABSOLUTE     
            XDATA   E6ADH     0001H     ABSOLUTE     
            XDATA   E6AEH     0001H     ABSOLUTE     
            XDATA   E6AFH     0001H     ABSOLUTE     
            XDATA   E6B0H     0001H     ABSOLUTE     
            XDATA   E6B1H     0001H     ABSOLUTE     
            XDATA   E6B2H     0001H     ABSOLUTE     
            XDATA   E6B3H     0001H     ABSOLUTE     
            XDATA   E6B4H     0001H     ABSOLUTE     
            XDATA   E6B5H     0001H     ABSOLUTE     
                    E6B6H     0002H                  *** GAP ***
            XDATA   E6B8H     0008H     ABSOLUTE     
            XDATA   E6C0H     0001H     ABSOLUTE     
            XDATA   E6C1H     0001H     ABSOLUTE     
            XDATA   E6C2H     0001H     ABSOLUTE     
            XDATA   E6C3H     0001H     ABSOLUTE     
            XDATA   E6C4H     0001H     ABSOLUTE     
            XDATA   E6C5H     0001H     ABSOLUTE     
            XDATA   E6C6H     0001H     ABSOLUTE     
            XDATA   E6C7H     0001H     ABSOLUTE     
            XDATA   E6C8H     0001H     ABSOLUTE     
            XDATA   E6C9H     0001H     ABSOLUTE     
            XDATA   E6CAH     0001H     ABSOLUTE     
            XDATA   E6CBH     0001H     ABSOLUTE     
            XDATA   E6CCH     0001H     ABSOLUTE     
            XDATA   E6CDH     0001H     ABSOLUTE     
            XDATA   E6CEH     0001H     ABSOLUTE     
            XDATA   E6CFH     0001H     ABSOLUTE     
            XDATA   E6D0H     0001H     ABSOLUTE     
            XDATA   E6D1H     0001H     ABSOLUTE     
            XDATA   E6D2H     0001H     ABSOLUTE     
            XDATA   E6D3H     0001H     ABSOLUTE     
            XDATA   E6D4H     0001H     ABSOLUTE     
                    E6D5H     0005H                  *** GAP ***
            XDATA   E6DAH     0001H     ABSOLUTE     
            XDATA   E6DBH     0001H     ABSOLUTE     
            XDATA   E6DCH     0001H     ABSOLUTE     
BL51 BANKED LINKER/LOCATER V6.02                                                      04/19/2018  15:18:09  PAGE 5


                    E6DDH     0005H                  *** GAP ***
            XDATA   E6E2H     0001H     ABSOLUTE     
            XDATA   E6E3H     0001H     ABSOLUTE     
            XDATA   E6E4H     0001H     ABSOLUTE     
                    E6E5H     0005H                  *** GAP ***
            XDATA   E6EAH     0001H     ABSOLUTE     
            XDATA   E6EBH     0001H     ABSOLUTE     
            XDATA   E6ECH     0001H     ABSOLUTE     
                    E6EDH     0003H                  *** GAP ***
            XDATA   E6F0H     0001H     ABSOLUTE     
            XDATA   E6F1H     0001H     ABSOLUTE     
            XDATA   E6F2H     0001H     ABSOLUTE     
            XDATA   E6F3H     0001H     ABSOLUTE     
            XDATA   E6F4H     0001H     ABSOLUTE     
            XDATA   E6F5H     0001H     ABSOLUTE     
                    E6F6H     0002H                  *** GAP ***
            XDATA   E6F8H     0001H     ABSOLUTE     
            XDATA   E6F9H     0001H     ABSOLUTE     
            XDATA   E6FAH     0001H     ABSOLUTE     
            XDATA   E6FBH     0001H     ABSOLUTE     
            XDATA   E6FCH     0001H     ABSOLUTE     
            XDATA   E6FDH     0001H     ABSOLUTE     
            XDATA   E6FEH     0001H     ABSOLUTE     
                    E6FFH     0041H                  *** GAP ***
            XDATA   E740H     0040H     ABSOLUTE     
            XDATA   E780H     0040H     ABSOLUTE     
            XDATA   E7C0H     0040H     ABSOLUTE     
                    E800H     0800H                  *** GAP ***
            XDATA   F000H     0400H     ABSOLUTE     
            XDATA   F400H     0400H     ABSOLUTE     
            XDATA   F800H     0400H     ABSOLUTE     
            XDATA   FC00H     0400H     ABSOLUTE     

            * * * * * * *   C O D E   M E M O R Y   * * * * * * *
            CODE    0000H     0003H     ABSOLUTE     
                    0003H     0008H                  *** GAP ***
            CODE    000BH     0003H     ABSOLUTE     
                    000EH     000DH                  *** GAP ***
            CODE    001BH     0003H     ABSOLUTE     
                    001EH     0015H                  *** GAP ***
            CODE    0033H     0003H     ABSOLUTE     
                    0036H     000DH                  *** GAP ***
            CODE    0043H     0003H     ABSOLUTE     
                    0046H     000DH                  *** GAP ***
            CODE    0053H     0003H     ABSOLUTE     
                    0056H     002AH                  *** GAP ***
            CODE    0080H     0316H     UNIT         ?PR?TD_POLL?PEDALERA
            CODE    0396H     02DFH     UNIT         ?PR?DR_VENDORCMND?PEDALERA
            CODE    0675H     0237H     UNIT         ?PR?SETUPCOMMAND?FW
            CODE    08ACH     0167H     UNIT         ?PR?MAIN?FW
            CODE    0A13H     009FH     UNIT         ?PR?_ANTIREBOTEPEDALES?PEDALERA
            CODE    0AB2H     0046H     UNIT         ?PR?_EZUSB_DELAY?DELAY
            CODE    0AF8H     0008H     UNIT         ?PR?DR_SETCONFIGURATION?PEDALERA
            CODE    0B00H     00B8H     PAGE         ?PR?USB_JUMP_TABLE?USBJT
            CODE    0BB8H     008CH     UNIT         ?C_C51STARTUP
            CODE    0C44H     0052H     UNIT         ?PR?_I2CWRITE?I2C
            CODE    0C96H     0043H     UNIT         ?PR?ISR_URES?PEDALERA
BL51 BANKED LINKER/LOCATER V6.02                                                      04/19/2018  15:18:09  PAGE 6


            CODE    0CD9H     0025H     UNIT         EZUSB
            CODE    0CFEH     0002H     UNIT         ?PR?TD_SUSPEND?PEDALERA
            CODE    0D00H     0072H     PAGE         DSCR
            CODE    0D72H     0043H     UNIT         ?PR?ISR_HIGHSPEED?PEDALERA
            CODE    0DB5H     003DH     UNIT         ?C_INITSEG
            CODE    0DF2H     0039H     UNIT         ?PR?TIMER1?INTERRUPCIONES
            CODE    0E2BH     0037H     UNIT         ?C?LIB_CODE
            CODE    0E62H     002FH     UNIT         ?PR?EZUSB_DISCON?DISCON
            CODE    0E91H     002CH     UNIT         ?PR?EZUSB_RESUME?RESUME
            CODE    0EBDH     002BH     UNIT         ?PR?_EZUSB_GETSTRINGDSCR?GET_STRD
            CODE    0EE8H     0025H     UNIT         ?PR?INICIALIZARPUERTOS?PEDALERA
            CODE    0F0DH     0022H     UNIT         ?PR?_SETDAC5571?I2C
            CODE    0F2FH     0021H     UNIT         ?PR?TIMER0?INTERRUPCIONES
            CODE    0F50H     0021H     UNIT         ?PR?TIMER0_INIT?PEDALERA
            CODE    0F71H     0021H     UNIT         ?PR?TIMER1_INIT?PEDALERA
            CODE    0F92H     001FH     UNIT         ?PR?ISR_SUDAV?PEDALERA
            CODE    0FB1H     0018H     UNIT         ?PR?ISR_SUSP?PEDALERA
            CODE    0FC9H     0016H     UNIT         ?PR?ISR_SUTOK?PEDALERA
            CODE    0FDFH     0016H     UNIT         ?PR?ISR_SOF?PEDALERA
            CODE    0FF5H     0016H     UNIT         ?PR?I2CWAITFORACK?I2C
            CODE    100BH     0012H     UNIT         ?PR?TD_INIT?PEDALERA
            CODE    101DH     0012H     UNIT         ?PR?DR_GETCONFIGURATION?PEDALERA
            CODE    102FH     0012H     UNIT         ?PR?DR_GETINTERFACE?PEDALERA
            CODE    1041H     000EH     UNIT         ?PR?_I2CSTARTANDADDRW?I2C
            CODE    104FH     000BH     UNIT         ?PR?HIGHSPEEDCAPABLE?FW
            CODE    105AH     000AH     UNIT         ?CO?FW
            CODE    1064H     0008H     UNIT         ?PR?DR_SETINTERFACE?PEDALERA
            CODE    106CH     0008H     UNIT         ?PR?I2CWAITFORSTOP?I2C
            CODE    1074H     0004H     UNIT         ?PR?RESUME_ISR?FW
            CODE    1078H     0002H     UNIT         ?PR?TD_RESUME?PEDALERA
            CODE    107AH     0002H     UNIT         ?PR?DR_GETDESCRIPTOR?PEDALERA
            CODE    107CH     0002H     UNIT         ?PR?DR_GETSTATUS?PEDALERA
            CODE    107EH     0002H     UNIT         ?PR?DR_CLEARFEATURE?PEDALERA
            CODE    1080H     0002H     UNIT         ?PR?DR_SETFEATURE?PEDALERA
            CODE    1082H     0001H     UNIT         ?PR?ISR_EP0ACK?PEDALERA
            CODE    1083H     0001H     UNIT         ?PR?ISR_STUB?PEDALERA
            CODE    1084H     0001H     UNIT         ?PR?ISR_EP0IN?PEDALERA
            CODE    1085H     0001H     UNIT         ?PR?ISR_EP0OUT?PEDALERA
            CODE    1086H     0001H     UNIT         ?PR?ISR_EP1IN?PEDALERA
            CODE    1087H     0001H     UNIT         ?PR?ISR_EP1OUT?PEDALERA
            CODE    1088H     0001H     UNIT         ?PR?ISR_EP2INOUT?PEDALERA
            CODE    1089H     0001H     UNIT         ?PR?ISR_EP4INOUT?PEDALERA
            CODE    108AH     0001H     UNIT         ?PR?ISR_EP6INOUT?PEDALERA
            CODE    108BH     0001H     UNIT         ?PR?ISR_EP8INOUT?PEDALERA
            CODE    108CH     0001H     UNIT         ?PR?ISR_IBN?PEDALERA
            CODE    108DH     0001H     UNIT         ?PR?ISR_EP0PINGNAK?PEDALERA
            CODE    108EH     0001H     UNIT         ?PR?ISR_EP1PINGNAK?PEDALERA
            CODE    108FH     0001H     UNIT         ?PR?ISR_EP2PINGNAK?PEDALERA
            CODE    1090H     0001H     UNIT         ?PR?ISR_EP4PINGNAK?PEDALERA
            CODE    1091H     0001H     UNIT         ?PR?ISR_EP6PINGNAK?PEDALERA
            CODE    1092H     0001H     UNIT         ?PR?ISR_EP8PINGNAK?PEDALERA
            CODE    1093H     0001H     UNIT         ?PR?ISR_ERRORLIMIT?PEDALERA
            CODE    1094H     0001H     UNIT         ?PR?ISR_EP2PIDERROR?PEDALERA
            CODE    1095H     0001H     UNIT         ?PR?ISR_EP4PIDERROR?PEDALERA
            CODE    1096H     0001H     UNIT         ?PR?ISR_EP6PIDERROR?PEDALERA
            CODE    1097H     0001H     UNIT         ?PR?ISR_EP8PIDERROR?PEDALERA
            CODE    1098H     0001H     UNIT         ?PR?ISR_EP2PFLAG?PEDALERA
BL51 BANKED LINKER/LOCATER V6.02                                                      04/19/2018  15:18:09  PAGE 7


            CODE    1099H     0001H     UNIT         ?PR?ISR_EP4PFLAG?PEDALERA
            CODE    109AH     0001H     UNIT         ?PR?ISR_EP6PFLAG?PEDALERA
            CODE    109BH     0001H     UNIT         ?PR?ISR_EP8PFLAG?PEDALERA
            CODE    109CH     0001H     UNIT         ?PR?ISR_EP2EFLAG?PEDALERA
            CODE    109DH     0001H     UNIT         ?PR?ISR_EP4EFLAG?PEDALERA
            CODE    109EH     0001H     UNIT         ?PR?ISR_EP6EFLAG?PEDALERA
            CODE    109FH     0001H     UNIT         ?PR?ISR_EP8EFLAG?PEDALERA
            CODE    10A0H     0001H     UNIT         ?PR?ISR_EP2FFLAG?PEDALERA
            CODE    10A1H     0001H     UNIT         ?PR?ISR_EP4FFLAG?PEDALERA
            CODE    10A2H     0001H     UNIT         ?PR?ISR_EP6FFLAG?PEDALERA
            CODE    10A3H     0001H     UNIT         ?PR?ISR_EP8FFLAG?PEDALERA
            CODE    10A4H     0001H     UNIT         ?PR?ISR_GPIFCOMPLETE?PEDALERA
            CODE    10A5H     0001H     UNIT         ?PR?ISR_GPIFWAVEFORM?PEDALERA



OVERLAY MAP OF MODULE:   InterfazPedalera (FW)


SEGMENT                                      BIT_GROUP          DATA_GROUP          XDATA_GROUP
  +--> CALLED SEGMENT                     START    LENGTH     START    LENGTH     START    LENGTH
-------------------------------------------------------------------------------------------------
?PR?USB_JUMP_TABLE?USBJT                  -----    -----      -----    -----      -----    -----
  +--> ?PR?ISR_SUDAV?PEDALERA
  +--> ?PR?ISR_SOF?PEDALERA
  +--> ?PR?ISR_SUTOK?PEDALERA
  +--> ?PR?ISR_SUSP?PEDALERA
  +--> ?PR?ISR_URES?PEDALERA
  +--> ?PR?ISR_HIGHSPEED?PEDALERA
  +--> ?PR?ISR_EP0ACK?PEDALERA
  +--> ?PR?ISR_STUB?PEDALERA
  +--> ?PR?ISR_EP0IN?PEDALERA
  +--> ?PR?ISR_EP0OUT?PEDALERA
  +--> ?PR?ISR_EP1IN?PEDALERA
  +--> ?PR?ISR_EP1OUT?PEDALERA
  +--> ?PR?ISR_EP2INOUT?PEDALERA
  +--> ?PR?ISR_EP4INOUT?PEDALERA
  +--> ?PR?ISR_EP6INOUT?PEDALERA
  +--> ?PR?ISR_EP8INOUT?PEDALERA
  +--> ?PR?ISR_IBN?PEDALERA
  +--> ?PR?ISR_EP0PINGNAK?PEDALERA
  +--> ?PR?ISR_EP1PINGNAK?PEDALERA
  +--> ?PR?ISR_EP2PINGNAK?PEDALERA
  +--> ?PR?ISR_EP4PINGNAK?PEDALERA
  +--> ?PR?ISR_EP6PINGNAK?PEDALERA
  +--> ?PR?ISR_EP8PINGNAK?PEDALERA
  +--> ?PR?ISR_ERRORLIMIT?PEDALERA
  +--> ?PR?ISR_EP2PIDERROR?PEDALERA
  +--> ?PR?ISR_EP4PIDERROR?PEDALERA
  +--> ?PR?ISR_EP6PIDERROR?PEDALERA
  +--> ?PR?ISR_EP8PIDERROR?PEDALERA
  +--> ?PR?ISR_EP2PFLAG?PEDALERA
  +--> ?PR?ISR_EP4PFLAG?PEDALERA
  +--> ?PR?ISR_EP6PFLAG?PEDALERA
  +--> ?PR?ISR_EP8PFLAG?PEDALERA
  +--> ?PR?ISR_EP2EFLAG?PEDALERA
  +--> ?PR?ISR_EP4EFLAG?PEDALERA
BL51 BANKED LINKER/LOCATER V6.02                                                      04/19/2018  15:18:09  PAGE 8


  +--> ?PR?ISR_EP6EFLAG?PEDALERA
  +--> ?PR?ISR_EP8EFLAG?PEDALERA
  +--> ?PR?ISR_EP2FFLAG?PEDALERA
  +--> ?PR?ISR_EP4FFLAG?PEDALERA
  +--> ?PR?ISR_EP6FFLAG?PEDALERA
  +--> ?PR?ISR_EP8FFLAG?PEDALERA
  +--> ?PR?ISR_GPIFCOMPLETE?PEDALERA
  +--> ?PR?ISR_GPIFWAVEFORM?PEDALERA

*** NEW ROOT ***************************************************

?C_C51STARTUP                             -----    -----      -----    -----      -----    -----
  +--> ?PR?MAIN?FW
  +--> ?C_INITSEG

?PR?MAIN?FW                               -----    -----      0008H    0010H      -----    -----
  +--> ?PR?TD_INIT?PEDALERA
  +--> ?PR?EZUSB_DISCON?DISCON
  +--> ?PR?TD_POLL?PEDALERA
  +--> ?PR?SETUPCOMMAND?FW
  +--> ?PR?TD_SUSPEND?PEDALERA
  +--> ?PR?EZUSB_RESUME?RESUME
  +--> ?PR?TD_RESUME?PEDALERA

?PR?TD_INIT?PEDALERA                      -----    -----      -----    -----      -----    -----
  +--> ?PR?INICIALIZARPUERTOS?PEDALERA
  +--> ?PR?TIMER0_INIT?PEDALERA
  +--> ?PR?TIMER1_INIT?PEDALERA

?PR?EZUSB_DISCON?DISCON                   0020H.5  0000H.1    -----    -----      -----    -----
  +--> ?PR?_EZUSB_DELAY?DELAY

?PR?_EZUSB_DELAY?DELAY                    -----    -----      0018H    0002H      -----    -----

?PR?TD_POLL?PEDALERA                      -----    -----      -----    -----      -----    -----
  +--> ?PR?_ANTIREBOTEPEDALES?PEDALERA

?PR?_ANTIREBOTEPEDALES?PEDALERA           0020H.5  0000H.1    -----    -----      -----    -----

?PR?SETUPCOMMAND?FW                       -----    -----      -----    -----      -----    -----
  +--> ?PR?DR_GETDESCRIPTOR?PEDALERA
  +--> ?PR?HIGHSPEEDCAPABLE?FW
  +--> ?PR?_EZUSB_GETSTRINGDSCR?GET_STRD
  +--> ?PR?DR_GETINTERFACE?PEDALERA
  +--> ?PR?DR_SETINTERFACE?PEDALERA
  +--> ?PR?DR_SETCONFIGURATION?PEDALERA
  +--> ?PR?DR_GETCONFIGURATION?PEDALERA
  +--> ?PR?DR_GETSTATUS?PEDALERA
  +--> ?CO?FW
  +--> ?PR?DR_CLEARFEATURE?PEDALERA
  +--> ?PR?DR_SETFEATURE?PEDALERA
  +--> ?PR?DR_VENDORCMND?PEDALERA

?PR?DR_VENDORCMND?PEDALERA                -----    -----      -----    -----      -----    -----
  +--> ?PR?_SETDAC5571?I2C

?PR?_SETDAC5571?I2C                       -----    -----      -----    -----      2000H    0002H
BL51 BANKED LINKER/LOCATER V6.02                                                      04/19/2018  15:18:09  PAGE 9


  +--> ?PR?_I2CWRITE?I2C

?PR?_I2CWRITE?I2C                         -----    -----      0018H    0005H      -----    -----
  +--> ?PR?I2CWAITFORSTOP?I2C
  +--> ?PR?_I2CSTARTANDADDRW?I2C
  +--> ?PR?I2CWAITFORACK?I2C

?PR?EZUSB_RESUME?RESUME                   -----    -----      -----    -----      -----    -----
  +--> ?PR?_EZUSB_DELAY?DELAY



SYMBOL TABLE OF MODULE:  InterfazPedalera (FW)

  VALUE           TYPE          NAME
  ----------------------------------

  -------         MODULE        FW
  C:0000H         SYMBOL        _ICE_DUMMY_
  B:00A8H.7       PUBLIC        EA
  B:0020H.0       PUBLIC        Rwuen
  B:0020H.1       PUBLIC        GotSUD
  C:105AH         PUBLIC        EPCS_Offset_Lookup_Table
  C:104FH         PUBLIC        HighSpeedCapable
  C:08ACH         PUBLIC        main
  B:00E8H.0       PUBLIC        EUSB
  C:1074H         PUBLIC        resume_isr
  D:003FH         PUBLIC        pHighSpeedConfigDscr
  D:0041H         PUBLIC        pDeviceDscr
  C:0675H         PUBLIC        SetupCommand
  D:0043H         PUBLIC        pConfigDscr
  D:0045H         PUBLIC        pOtherConfigDscr
  D:0047H         PUBLIC        pFullSpeedConfigDscr
  B:0020H.2       PUBLIC        Selfpwr
  D:0049H         PUBLIC        pDeviceQualDscr
  D:00D8H         PUBLIC        EICON
  D:008EH         PUBLIC        CKCON
  D:004BH         PUBLIC        pStringDscr
  B:0020H.3       PUBLIC        Sleep
  -------         PROC          MAIN
  -------         DO            
  D:0008H         SYMBOL        i
  D:0006H         SYMBOL        offset
  D:000CH         SYMBOL        DevDescrLen
  D:0010H         SYMBOL        j
  D:0014H         SYMBOL        IntDescrAddr
  D:0016H         SYMBOL        ExtDescrAddr
  -------         ENDDO         
  C:08ACH         LINE#         88
  C:08ACH         LINE#         89
  C:08ACH         LINE#         93
  C:08B5H         LINE#         98
  C:08B7H         LINE#         99
  C:08B9H         LINE#         100
  C:08BBH         LINE#         101
  C:08BDH         LINE#         104
  C:08C0H         LINE#         113
BL51 BANKED LINKER/LOCATER V6.02                                                      04/19/2018  15:18:09  PAGE 10


  C:08C8H         LINE#         114
  C:08CEH         LINE#         115
  C:08D4H         LINE#         116
  C:08DAH         LINE#         117
  C:08E0H         LINE#         124
  C:08E8H         LINE#         125
  C:08E8H         LINE#         127
  C:08EEH         LINE#         128
  C:08F2H         LINE#         129
  C:090AH         LINE#         130
  C:0928H         LINE#         131
  C:095BH         LINE#         134
  C:0961H         LINE#         135
  C:096BH         LINE#         136
  C:0976H         LINE#         137
  C:0981H         LINE#         138
  C:098CH         LINE#         139
  C:0997H         LINE#         140
  C:09A2H         LINE#         141
  C:09ADH         LINE#         142
  C:09ADH         LINE#         144
  C:09AFH         LINE#         145
  C:09B2H         LINE#         147
  C:09B9H         LINE#         149
  C:09C0H         LINE#         150
  C:09C2H         LINE#         156
  C:09C9H         LINE#         157
  C:09C9H         LINE#         158
  C:09CEH         LINE#         159
  C:09CEH         LINE#         165
  C:09D5H         LINE#         167
  C:09D8H         LINE#         170
  C:09DAH         LINE#         173
  C:09DAH         LINE#         174
  C:09DAH         LINE#         176
  C:09DDH         LINE#         179
  C:09E0H         LINE#         180
  C:09E0H         LINE#         181
  C:09E3H         LINE#         182
  C:09E5H         LINE#         183
  C:09E5H         LINE#         190
  C:09E8H         LINE#         191
  C:09E8H         LINE#         192
  C:09EDH         LINE#         193
  C:09EDH         LINE#         194
  C:09EFH         LINE#         196
  C:09EFH         LINE#         197
  C:09F2H         LINE#         198
  C:09F2H         LINE#         199
  C:0A0BH         LINE#         204
  C:0A0EH         LINE#         205
  C:0A11H         LINE#         206
  C:0A11H         LINE#         207
  C:0A11H         LINE#         209
  -------         ENDPROC       MAIN
  -------         PROC          HIGHSPEEDCAPABLE
  C:104FH         LINE#         212
BL51 BANKED LINKER/LOCATER V6.02                                                      04/19/2018  15:18:09  PAGE 11


  C:104FH         LINE#         213
  C:104FH         LINE#         218
  C:1056H         LINE#         219
  C:1058H         LINE#         221
  C:1059H         LINE#         222
  -------         ENDPROC       HIGHSPEEDCAPABLE
  -------         PROC          SETUPCOMMAND
  -------         DO            
  D:0001H         SYMBOL        dscr_ptr
  -------         ENDDO         
  C:0675H         LINE#         225
  C:0675H         LINE#         226
  C:0675H         LINE#         229
  C:06ABH         LINE#         230
  C:06ABH         LINE#         231
  C:06ABH         LINE#         232
  C:06B3H         LINE#         233
  C:06C9H         LINE#         234
  C:06C9H         LINE#         235
  C:06C9H         LINE#         236
  C:06CFH         LINE#         237
  C:06D1H         LINE#         238
  C:06D3H         LINE#         239
  C:06D3H         LINE#         242
  C:06D8H         LINE#         243
  C:06D8H         LINE#         244
  C:06DEH         LINE#         245
  C:06E0H         LINE#         246
  C:06E2H         LINE#         252
  C:06E2H         LINE#         253
  C:06E8H         LINE#         254
  C:06EAH         LINE#         255
  C:06ECH         LINE#         256
  C:06ECH         LINE#         257
  C:06F2H         LINE#         258
  C:06F4H         LINE#         259
  C:06F6H         LINE#         260
  C:06F6H         LINE#         261
  C:0709H         LINE#         262
  C:0709H         LINE#         263
  C:070EH         LINE#         264
  C:0713H         LINE#         265
  C:0716H         LINE#         267
  C:0716H         LINE#         268
  C:0719H         LINE#         269
  C:0719H         LINE#         270
  C:0719H         LINE#         271
  C:0719H         LINE#         272
  C:071CH         LINE#         273
  C:071CH         LINE#         274
  C:071FH         LINE#         275
  C:0722H         LINE#         276
  C:0722H         LINE#         277
  C:0725H         LINE#         278
  C:0728H         LINE#         279
  C:0728H         LINE#         280
  C:072BH         LINE#         281
BL51 BANKED LINKER/LOCATER V6.02                                                      04/19/2018  15:18:09  PAGE 12


  C:072EH         LINE#         282
  C:072EH         LINE#         283
  C:0731H         LINE#         284
  C:0734H         LINE#         285
  C:0734H         LINE#         286
  C:073CH         LINE#         287
  C:074BH         LINE#         288
  C:074BH         LINE#         289
  C:074BH         LINE#         290
  C:0757H         LINE#         291
  C:0757H         LINE#         292
  C:0757H         LINE#         293
  C:0757H         LINE#         294
  C:0759H         LINE#         295
  C:0759H         LINE#         296
  C:075EH         LINE#         297
  C:075EH         LINE#         298
  C:075EH         LINE#         299
  C:075EH         LINE#         300
  C:0760H         LINE#         301
  C:0760H         LINE#         302
  C:079EH         LINE#         303
  C:07A1H         LINE#         304
  C:07A5H         LINE#         305
  C:07ABH         LINE#         306
  C:07AEH         LINE#         307
  C:07AEH         LINE#         308
  C:07AEH         LINE#         309
  C:07AEH         LINE#         310
  C:07B1H         LINE#         311
  C:07B1H         LINE#         312
  C:07B9H         LINE#         313
  C:07C8H         LINE#         314
  C:07C8H         LINE#         315
  C:07C8H         LINE#         316
  C:07CFH         LINE#         317
  C:07D4H         LINE#         319
  C:07D4H         LINE#         320
  C:07D7H         LINE#         321
  C:07D7H         LINE#         322
  C:07DDH         LINE#         323
  C:07DDH         LINE#         324
  C:0818H         LINE#         325
  C:0830H         LINE#         326
  C:0832H         LINE#         328
  C:0832H         LINE#         329
  C:0834H         LINE#         330
  C:0834H         LINE#         331
  C:0834H         LINE#         332
  C:0834H         LINE#         333
  C:0839H         LINE#         334
  C:0845H         LINE#         335
  C:0845H         LINE#         336
  C:0845H         LINE#         337
  C:084CH         LINE#         338
  C:0850H         LINE#         339
  C:0858H         LINE#         345
BL51 BANKED LINKER/LOCATER V6.02                                                      04/19/2018  15:18:09  PAGE 13


  C:0858H         LINE#         347
  C:0858H         LINE#         348
  C:085AH         LINE#         349
  C:085AH         LINE#         350
  C:0891H         LINE#         351
  C:0893H         LINE#         352
  C:0893H         LINE#         353
  C:0896H         LINE#         354
  C:0896H         LINE#         355
  C:0898H         LINE#         356
  C:0898H         LINE#         357
  C:089DH         LINE#         358
  C:08A4H         LINE#         359
  C:08A4H         LINE#         362
  C:08ABH         LINE#         363
  -------         ENDPROC       SETUPCOMMAND
  -------         PROC          RESUME_ISR
  C:1074H         LINE#         366
  C:1074H         LINE#         368
  C:1077H         LINE#         369
  -------         ENDPROC       RESUME_ISR
  -------         ENDMOD        FW

  -------         MODULE        DSCR
  C:0D00H         SEGMENT       DSCR
  C:0D00H         PUBLIC        DEVICEDSCR
  C:0D12H         PUBLIC        DEVICEQUALDSCR
  C:0D35H         PUBLIC        FULLSPEEDCONFIGDSCR
  C:0D1CH         PUBLIC        HIGHSPEEDCONFIGDSCR
  C:0D4EH         PUBLIC        STRINGDSCR
  C:0D70H         PUBLIC        USERDSCR
  N:0002H         SYMBOL        DSCR_CONFIG
  N:0009H         SYMBOL        DSCR_CONFIG_LEN
  N:0001H         SYMBOL        DSCR_DEVICE
  N:0012H         SYMBOL        DSCR_DEVICE_LEN
  N:0006H         SYMBOL        DSCR_DEVQUAL
  N:000AH         SYMBOL        DSCR_DEVQUAL_LEN
  N:0005H         SYMBOL        DSCR_ENDPNT
  N:0007H         SYMBOL        DSCR_ENDPNT_LEN
  N:0004H         SYMBOL        DSCR_INTRFC
  N:0009H         SYMBOL        DSCR_INTRFC_LEN
  N:0003H         SYMBOL        DSCR_STRING
  N:0002H         SYMBOL        ET_BULK
  N:0000H         SYMBOL        ET_CONTROL
  N:0003H         SYMBOL        ET_INT
  N:0001H         SYMBOL        ET_ISO
  C:0D4EH         SYMBOL        FULLSPEEDCONFIGDSCREND
  C:0D35H         SYMBOL        HIGHSPEEDCONFIGDSCREND
  C:0D4EH         SYMBOL        STRINGDSCR0
  C:0D52H         SYMBOL        STRINGDSCR0END
  C:0D52H         SYMBOL        STRINGDSCR1
  C:0D62H         SYMBOL        STRINGDSCR1END
  C:0D62H         SYMBOL        STRINGDSCR2
  C:0D70H         SYMBOL        STRINGDSCR2END
  -------         ENDMOD        DSCR

  -------         MODULE        RESUME
BL51 BANKED LINKER/LOCATER V6.02                                                      04/19/2018  15:18:09  PAGE 14


  C:0000H         SYMBOL        _ICE_DUMMY_
  C:0E91H         PUBLIC        EZUSB_Resume
  -------         PROC          EZUSB_RESUME
  C:0E91H         LINE#         38
  C:0E91H         LINE#         39
  C:0E91H         LINE#         40
  C:0EA7H         LINE#         42
  C:0EA7H         LINE#         43
  C:0EAEH         LINE#         44
  C:0EB5H         LINE#         45
  C:0EBCH         LINE#         46
  C:0EBCH         LINE#         47
  -------         ENDPROC       EZUSB_RESUME
  -------         ENDMOD        RESUME

  -------         MODULE        DISCON
  C:0000H         SYMBOL        _ICE_DUMMY_
  D:0091H         PUBLIC        EXIF
  C:0E62H         PUBLIC        EZUSB_Discon
  -------         PROC          EZUSB_DISCON
  B:0020H.5       SYMBOL        renum
  C:0E62H         LINE#         39
  C:0E62H         LINE#         40
  C:0E62H         LINE#         42
  C:0E65H         LINE#         43
  C:0E6EH         LINE#         45
  C:0E75H         LINE#         47
  C:0E7CH         LINE#         49
  C:0E82H         LINE#         50
  C:0E86H         LINE#         51
  C:0E89H         LINE#         53
  C:0E90H         LINE#         54
  -------         ENDPROC       EZUSB_DISCON
  -------         ENDMOD        DISCON

  -------         MODULE        EZREGS
  C:0000H         SYMBOL        _ICE_DUMMY_
  X:E652H         PUBLIC        EP4FIFOIE
  X:E668H         PUBLIC        INTSETUP
  X:E600H         PUBLIC        CPUCS
  X:E654H         PUBLIC        EP6FIFOIE
  X:E680H         PUBLIC        USBCS
  X:E65FH         PUBLIC        EPIRQ
  X:E656H         PUBLIC        EP8FIFOIE
  X:E6F2H         PUBLIC        XGPIFSGLDATLNOX
  X:E6C0H         PUBLIC        GPIFWFSELECT
  X:E6F0H         PUBLIC        XGPIFSGLDATH
  X:E605H         PUBLIC        BREAKPT
  X:E609H         PUBLIC        FIFOPINPOLAR
  X:E640H         PUBLIC        EP2ISOINPKTS
  X:E678H         PUBLIC        I2CS
  X:E610H         PUBLIC        EP1OUTCFG
  X:E6F9H         PUBLIC        TESTCFG
  X:E641H         PUBLIC        EP4ISOINPKTS
  X:E68AH         PUBLIC        EP0BCH
  X:E661H         PUBLIC        GPIFIRQ
  X:E642H         PUBLIC        EP6ISOINPKTS
BL51 BANKED LINKER/LOCATER V6.02                                                      04/19/2018  15:18:09  PAGE 15


  X:E690H         PUBLIC        EP2BCH
  X:E643H         PUBLIC        EP8ISOINPKTS
  X:E694H         PUBLIC        EP4BCH
  X:E68BH         PUBLIC        EP0BCL
  X:E612H         PUBLIC        EP2CFG
  X:E698H         PUBLIC        EP6BCH
  X:E691H         PUBLIC        EP2BCL
  X:E613H         PUBLIC        EP4CFG
  X:E6A7H         PUBLIC        EP2FIFOFLGS
  X:E69CH         PUBLIC        EP8BCH
  X:E695H         PUBLIC        EP4BCL
  X:E628H         PUBLIC        ECCCFG
  X:E614H         PUBLIC        EP6CFG
  X:E6A8H         PUBLIC        EP4FIFOFLGS
  X:E699H         PUBLIC        EP6BCL
  X:E780H         PUBLIC        EP1OUTBUF
  X:E67BH         PUBLIC        XAUTODAT1
  X:E615H         PUBLIC        EP8CFG
  X:E6A9H         PUBLIC        EP6FIFOFLGS
  X:E69DH         PUBLIC        EP8BCL
  X:E67CH         PUBLIC        XAUTODAT2
  X:E684H         PUBLIC        USBFRAMEH
  X:E6F5H         PUBLIC        GPIFABORT
  X:E6AAH         PUBLIC        EP8FIFOFLGS
  X:E6F8H         PUBLIC        DBUG
  X:E740H         PUBLIC        EP0BUF
  X:E6CBH         PUBLIC        FLOWSTB
  X:E65EH         PUBLIC        EPIE
  X:E685H         PUBLIC        USBFRAMEL
  X:E681H         PUBLIC        SUSPEND
  X:E60CH         PUBLIC        GPIFHOLDAMOUNT
  X:E6D4H         PUBLIC        EP2GPIFTRIG
  X:E6C7H         PUBLIC        FLOWLOGIC
  X:E6DCH         PUBLIC        EP4GPIFTRIG
  X:E604H         PUBLIC        FIFORESET
  X:E6E4H         PUBLIC        EP6GPIFTRIG
  X:E6C2H         PUBLIC        GPIFIDLECTL
  X:E6FAH         PUBLIC        USBTEST
  X:E6B3H         PUBLIC        SUDPTRH
  X:E6ECH         PUBLIC        EP8GPIFTRIG
  X:E6D2H         PUBLIC        EP2GPIFFLGSEL
  X:E611H         PUBLIC        EP1INCFG
  X:E6B4H         PUBLIC        SUDPTRL
  X:E687H         PUBLIC        FNADDR
  X:E6DAH         PUBLIC        EP4GPIFFLGSEL
  X:E6D1H         PUBLIC        GPIFTCB0
  X:E6CDH         PUBLIC        FLOWSTBHPERIOD
  X:E6D0H         PUBLIC        GPIFTCB1
  X:E665H         PUBLIC        CLRERRCNT
  X:E6E2H         PUBLIC        EP6GPIFFLGSEL
  X:E6CFH         PUBLIC        GPIFTCB2
  X:E664H         PUBLIC        ERRCNTLIM
  X:E6CEH         PUBLIC        GPIFTCB3
  X:E6EAH         PUBLIC        EP8GPIFFLGSEL
  X:E660H         PUBLIC        GPIFIE
  X:E67FH         PUBLIC        UDMACRCQUAL
  X:E400H         PUBLIC        GPIF_WAVE_DATA
BL51 BANKED LINKER/LOCATER V6.02                                                      04/19/2018  15:18:09  PAGE 16


  X:E6CCH         PUBLIC        FLOWSTBEDGE
  X:E6ABH         PUBLIC        EP2FIFOBCH
  X:E7C0H         PUBLIC        EP1INBUF
  X:E6C6H         PUBLIC        FLOWSTATE
  X:E6ADH         PUBLIC        EP4FIFOBCH
  X:E6CAH         PUBLIC        FLOWHOLDOFF
  X:E618H         PUBLIC        EP2FIFOCFG
  X:E6AFH         PUBLIC        EP6FIFOBCH
  X:E6ACH         PUBLIC        EP2FIFOBCL
  X:E619H         PUBLIC        EP4FIFOCFG
  X:E6B1H         PUBLIC        EP8FIFOBCH
  X:E6AEH         PUBLIC        EP4FIFOBCL
  X:E649H         PUBLIC        OUTPKTEND
  X:E663H         PUBLIC        USBERRIRQ
  X:E61AH         PUBLIC        EP6FIFOCFG
  X:E6B0H         PUBLIC        EP6FIFOBCL
  X:E620H         PUBLIC        EP2AUTOINLENH
  X:E61BH         PUBLIC        EP8FIFOCFG
  X:E6B2H         PUBLIC        EP8FIFOBCL
  X:E68DH         PUBLIC        EP1OUTBC
  X:E622H         PUBLIC        EP4AUTOINLENH
  X:E666H         PUBLIC        INT2IVEC
  X:E659H         PUBLIC        IBNIRQ
  X:E6FBH         PUBLIC        CT1
  X:E6C4H         PUBLIC        GPIFADRH
  X:E65BH         PUBLIC        NAKIRQ
  X:E624H         PUBLIC        EP6AUTOINLENH
  X:E621H         PUBLIC        EP2AUTOINLENL
  X:E601H         PUBLIC        IFCONFIG
  X:E6FCH         PUBLIC        CT2
  X:E6B5H         PUBLIC        SUDPTRCTL
  X:E667H         PUBLIC        INT4IVEC
  X:E6FDH         PUBLIC        CT3
  X:E67DH         PUBLIC        UDMACRCH
  X:E626H         PUBLIC        EP8AUTOINLENH
  X:E623H         PUBLIC        EP4AUTOINLENL
  X:E6FEH         PUBLIC        CT4
  X:F000H         PUBLIC        EP2FIFOBUF
  X:E6C5H         PUBLIC        GPIFADRL
  X:E625H         PUBLIC        EP6AUTOINLENL
  X:E630H         PUBLIC        EP2FIFOPFH
  X:F400H         PUBLIC        EP4FIFOBUF
  X:E67EH         PUBLIC        UDMACRCL
  X:E627H         PUBLIC        EP8AUTOINLENL
  X:E6D3H         PUBLIC        EP2GPIFPFSTOP
  X:E683H         PUBLIC        TOGCTL
  X:E632H         PUBLIC        EP4FIFOPFH
  X:F800H         PUBLIC        EP6FIFOBUF
  X:E629H         PUBLIC        ECCRESET
  X:E6DBH         PUBLIC        EP4GPIFPFSTOP
  X:E634H         PUBLIC        EP6FIFOPFH
  X:E631H         PUBLIC        EP2FIFOPFL
  X:FC00H         PUBLIC        EP8FIFOBUF
  X:E60BH         PUBLIC        REVCTL
  X:E6E3H         PUBLIC        EP6GPIFPFSTOP
  X:E636H         PUBLIC        EP8FIFOPFH
  X:E633H         PUBLIC        EP4FIFOPFL
BL51 BANKED LINKER/LOCATER V6.02                                                      04/19/2018  15:18:09  PAGE 17


  X:E608H         PUBLIC        UART230
  X:E480H         PUBLIC        RES_WAVEDATA_END
  X:E6EBH         PUBLIC        EP8GPIFPFSTOP
  X:E679H         PUBLIC        I2DAT
  X:E635H         PUBLIC        EP6FIFOPFL
  X:E6A1H         PUBLIC        EP1OUTCS
  X:E637H         PUBLIC        EP8FIFOPFL
  X:E65DH         PUBLIC        USBIRQ
  X:E670H         PUBLIC        PORTACFG
  X:E671H         PUBLIC        PORTCCFG
  X:E651H         PUBLIC        EP2FIFOIRQ
  X:E602H         PUBLIC        PINFLAGSAB
  X:E6A0H         PUBLIC        EP0CS
  X:E6F4H         PUBLIC        GPIFREADYSTAT
  X:E6C3H         PUBLIC        GPIFCTLCFG
  X:E672H         PUBLIC        PORTECFG
  X:E653H         PUBLIC        EP4FIFOIRQ
  X:E6C1H         PUBLIC        GPIFIDLECS
  X:E6A3H         PUBLIC        EP2CS
  X:E50DH         PUBLIC        GPCR2
  X:E67AH         PUBLIC        I2CTL
  X:E655H         PUBLIC        EP6FIFOIRQ
  X:E603H         PUBLIC        PINFLAGSCD
  X:E6A4H         PUBLIC        EP4CS
  X:E648H         PUBLIC        INPKTEND
  X:E657H         PUBLIC        EP8FIFOIRQ
  X:E6A5H         PUBLIC        EP6CS
  X:E6A6H         PUBLIC        EP8CS
  X:E68FH         PUBLIC        EP1INBC
  X:E662H         PUBLIC        USBERRIE
  X:E6C8H         PUBLIC        FLOWEQ0CTL
  X:E6C9H         PUBLIC        FLOWEQ1CTL
  X:E682H         PUBLIC        WAKEUPCS
  X:E6F1H         PUBLIC        XGPIFSGLDATLX
  X:E658H         PUBLIC        IBNIE
  X:E686H         PUBLIC        MICROFRAME
  X:E65AH         PUBLIC        NAKIE
  X:E6B8H         PUBLIC        SETUPDAT
  X:E62AH         PUBLIC        ECC1B0
  X:E62DH         PUBLIC        ECC2B0
  X:E62BH         PUBLIC        ECC1B1
  X:E6F3H         PUBLIC        GPIFREADYCFG
  X:E62EH         PUBLIC        ECC2B1
  X:E62CH         PUBLIC        ECC1B2
  X:E62FH         PUBLIC        ECC2B2
  X:E6A2H         PUBLIC        EP1INCS
  X:E606H         PUBLIC        BPADDRH
  X:E65CH         PUBLIC        USBIE
  X:E60AH         PUBLIC        REVID
  X:E607H         PUBLIC        BPADDRL
  X:E650H         PUBLIC        EP2FIFOIE
  -------         ENDMOD        EZREGS

  -------         MODULE        GET_STRD
  C:0000H         SYMBOL        _ICE_DUMMY_
  C:0EBDH         PUBLIC        _EZUSB_GetStringDscr
  -------         PROC          _EZUSB_GETSTRINGDSCR
BL51 BANKED LINKER/LOCATER V6.02                                                      04/19/2018  15:18:09  PAGE 18


  D:0001H         SYMBOL        StrIdx
  -------         DO            
  D:0006H         SYMBOL        dscr
  -------         ENDDO         
  C:0EBDH         LINE#         38
  C:0EBFH         LINE#         39
  C:0EBFH         LINE#         42
  C:0EC3H         LINE#         44
  C:0ECDH         LINE#         45
  C:0ECDH         LINE#         46
  C:0ED3H         LINE#         47
  C:0ED4H         LINE#         48
  C:0EE2H         LINE#         49
  C:0EE4H         LINE#         51
  C:0EE7H         LINE#         52
  -------         ENDPROC       _EZUSB_GETSTRINGDSCR
  -------         ENDMOD        GET_STRD

  -------         MODULE        SUSP
  C:0CD9H         SEGMENT       EZUSB
  C:0CD9H         PUBLIC        EZUSB_SUSP
  B:00D0H.6       SYMBOL        AC
  D:00E0H         SYMBOL        ACC
  D:009AH         SYMBOL        APTR1H
  D:009BH         SYMBOL        APTR1L
  D:009AH         SYMBOL        AUTOPTR1H
  D:009BH         SYMBOL        AUTOPTR1L
  D:009AH         SYMBOL        AUTOPTRH1
  D:009DH         SYMBOL        AUTOPTRH2
  D:009BH         SYMBOL        AUTOPTRL1
  D:009EH         SYMBOL        AUTOPTRL2
  D:00AFH         SYMBOL        AUTOPTRSETUP
  D:00F0H         SYMBOL        B
  X:E606H         SYMBOL        BPADDRH
  X:E607H         SYMBOL        BPADDRL
  X:E605H         SYMBOL        BREAKPT
  D:008EH         SYMBOL        CKCON
  X:E665H         SYMBOL        CLRERRCNT
  X:E600H         SYMBOL        CPUCS
  B:00C8H.0       SYMBOL        CP_RL2
  X:E6FBH         SYMBOL        CT1
  X:E6FCH         SYMBOL        CT2
  X:E6FDH         SYMBOL        CT3
  X:E6FEH         SYMBOL        CT4
  B:00D0H.7       SYMBOL        CY
  B:00C8H.1       SYMBOL        C_T2
  X:E6F8H         SYMBOL        DBUG
  D:0083H         SYMBOL        DPH
  D:0085H         SYMBOL        DPH1
  D:0082H         SYMBOL        DPL
  D:0084H         SYMBOL        DPL1
  D:0086H         SYMBOL        DPS
  B:00A8H.7       SYMBOL        EA
  X:E62AH         SYMBOL        ECC1B0
  X:E62BH         SYMBOL        ECC1B1
  X:E62CH         SYMBOL        ECC1B2
  X:E62DH         SYMBOL        ECC2B0
BL51 BANKED LINKER/LOCATER V6.02                                                      04/19/2018  15:18:09  PAGE 19


  X:E62EH         SYMBOL        ECC2B1
  X:E62FH         SYMBOL        ECC2B2
  X:E628H         SYMBOL        ECCCFG
  X:E629H         SYMBOL        ECCRESET
  B:00E8H.1       SYMBOL        EI2C
  D:00D8H         SYMBOL        EICON
  D:00E8H         SYMBOL        EIE
  B:00E8H.2       SYMBOL        EIEX4
  B:00E8H.3       SYMBOL        EIEX5
  B:00E8H.4       SYMBOL        EIEX6
  D:00F8H         SYMBOL        EIP
  B:00F8H.2       SYMBOL        EIPX4
  B:00F8H.3       SYMBOL        EIPX5
  B:00F8H.4       SYMBOL        EIPX6
  D:00BAH         SYMBOL        EP01STAT
  X:E68AH         SYMBOL        EP0BCH
  X:E68BH         SYMBOL        EP0BCL
  X:E740H         SYMBOL        EP0BUF
  X:E6A0H         SYMBOL        EP0CS
  X:E68FH         SYMBOL        EP1INBC
  X:E7C0H         SYMBOL        EP1INBUF
  X:E611H         SYMBOL        EP1INCFG
  X:E6A2H         SYMBOL        EP1INCS
  X:E68DH         SYMBOL        EP1OUTBC
  X:E780H         SYMBOL        EP1OUTBUF
  X:E610H         SYMBOL        EP1OUTCFG
  X:E6A1H         SYMBOL        EP1OUTCS
  D:00AAH         SYMBOL        EP2468STAT
  D:00ABH         SYMBOL        EP24FIFOFLGS
  X:E620H         SYMBOL        EP2AUTOINLENH
  X:E621H         SYMBOL        EP2AUTOINLENL
  X:E690H         SYMBOL        EP2BCH
  X:E691H         SYMBOL        EP2BCL
  X:E612H         SYMBOL        EP2CFG
  X:E6A3H         SYMBOL        EP2CS
  X:E6ABH         SYMBOL        EP2FIFOBCH
  X:E6ACH         SYMBOL        EP2FIFOBCL
  X:F000H         SYMBOL        EP2FIFOBUF
  X:E618H         SYMBOL        EP2FIFOCFG
  X:E6A7H         SYMBOL        EP2FIFOFLGS
  X:E650H         SYMBOL        EP2FIFOIE
  X:E651H         SYMBOL        EP2FIFOIRQ
  X:E630H         SYMBOL        EP2FIFOPFH
  X:E631H         SYMBOL        EP2FIFOPFL
  X:E6D2H         SYMBOL        EP2GPIFFLGSEL
  X:E6D3H         SYMBOL        EP2GPIFPFSTOP
  X:E6D0H         SYMBOL        EP2GPIFTCH
  X:E6D1H         SYMBOL        EP2GPIFTCL
  X:E6D4H         SYMBOL        EP2GPIFTRIG
  X:E640H         SYMBOL        EP2ISOINPKTS
  X:E622H         SYMBOL        EP4AUTOINLENH
  X:E623H         SYMBOL        EP4AUTOINLENL
  X:E694H         SYMBOL        EP4BCH
  X:E695H         SYMBOL        EP4BCL
  X:E613H         SYMBOL        EP4CFG
  X:E6A4H         SYMBOL        EP4CS
  X:E6ADH         SYMBOL        EP4FIFOBCH
BL51 BANKED LINKER/LOCATER V6.02                                                      04/19/2018  15:18:09  PAGE 20


  X:E6AEH         SYMBOL        EP4FIFOBCL
  X:F400H         SYMBOL        EP4FIFOBUF
  X:E619H         SYMBOL        EP4FIFOCFG
  X:E6A8H         SYMBOL        EP4FIFOFLGS
  X:E652H         SYMBOL        EP4FIFOIE
  X:E653H         SYMBOL        EP4FIFOIRQ
  X:E632H         SYMBOL        EP4FIFOPFH
  X:E633H         SYMBOL        EP4FIFOPFL
  X:E6DAH         SYMBOL        EP4GPIFFLGSEL
  X:E6DBH         SYMBOL        EP4GPIFPFSTOP
  X:E6D0H         SYMBOL        EP4GPIFTCH
  X:E6D1H         SYMBOL        EP4GPIFTCL
  X:E6DCH         SYMBOL        EP4GPIFTRIG
  X:E641H         SYMBOL        EP4ISOINPKTS
  D:00ACH         SYMBOL        EP68FIFOFLGS
  X:E624H         SYMBOL        EP6AUTOINLENH
  X:E625H         SYMBOL        EP6AUTOINLENL
  X:E698H         SYMBOL        EP6BCH
  X:E699H         SYMBOL        EP6BCL
  X:E614H         SYMBOL        EP6CFG
  X:E6A5H         SYMBOL        EP6CS
  X:E6AFH         SYMBOL        EP6FIFOBCH
  X:E6B0H         SYMBOL        EP6FIFOBCL
  X:F800H         SYMBOL        EP6FIFOBUF
  X:E61AH         SYMBOL        EP6FIFOCFG
  X:E6A9H         SYMBOL        EP6FIFOFLGS
  X:E654H         SYMBOL        EP6FIFOIE
  X:E655H         SYMBOL        EP6FIFOIRQ
  X:E634H         SYMBOL        EP6FIFOPFH
  X:E635H         SYMBOL        EP6FIFOPFL
  X:E6E2H         SYMBOL        EP6GPIFFLGSEL
  X:E6E3H         SYMBOL        EP6GPIFPFSTOP
  X:E6D0H         SYMBOL        EP6GPIFTCH
  X:E6D1H         SYMBOL        EP6GPIFTCL
  X:E6E4H         SYMBOL        EP6GPIFTRIG
  X:E642H         SYMBOL        EP6ISOINPKTS
  X:E626H         SYMBOL        EP8AUTOINLENH
  X:E627H         SYMBOL        EP8AUTOINLENL
  X:E69CH         SYMBOL        EP8BCH
  X:E69DH         SYMBOL        EP8BCL
  X:E615H         SYMBOL        EP8CFG
  X:E6A6H         SYMBOL        EP8CS
  X:E6B1H         SYMBOL        EP8FIFOBCH
  X:E6B2H         SYMBOL        EP8FIFOBCL
  X:FC00H         SYMBOL        EP8FIFOBUF
  X:E61BH         SYMBOL        EP8FIFOCFG
  X:E6AAH         SYMBOL        EP8FIFOFLGS
  X:E656H         SYMBOL        EP8FIFOIE
  X:E657H         SYMBOL        EP8FIFOIRQ
  X:E636H         SYMBOL        EP8FIFOPFH
  X:E637H         SYMBOL        EP8FIFOPFL
  X:E6EAH         SYMBOL        EP8GPIFFLGSEL
  X:E6EBH         SYMBOL        EP8GPIFPFSTOP
  X:E6D0H         SYMBOL        EP8GPIFTCH
  X:E6D1H         SYMBOL        EP8GPIFTCL
  X:E6ECH         SYMBOL        EP8GPIFTRIG
  X:E643H         SYMBOL        EP8ISOINPKTS
BL51 BANKED LINKER/LOCATER V6.02                                                      04/19/2018  15:18:09  PAGE 21


  X:E65EH         SYMBOL        EPIE
  X:E65FH         SYMBOL        EPIRQ
  B:00D8H.5       SYMBOL        ERESI
  X:E664H         SYMBOL        ERRCNTLIM
  C:0CECH         SYMBOL        ER_END
  B:00A8H.4       SYMBOL        ES0
  B:00A8H.6       SYMBOL        ES1
  B:00A8H.1       SYMBOL        ET0
  B:00A8H.3       SYMBOL        ET1
  B:00A8H.5       SYMBOL        ET2
  B:00E8H.0       SYMBOL        EUSB
  B:00A8H.0       SYMBOL        EX0
  B:00A8H.2       SYMBOL        EX1
  B:00C8H.3       SYMBOL        EXEN2
  B:00C8H.6       SYMBOL        EXF2
  D:0091H         SYMBOL        EXIF
  X:E67BH         SYMBOL        EXTAUTODAT1
  X:E67CH         SYMBOL        EXTAUTODAT2
  B:00D0H.5       SYMBOL        F0
  X:E609H         SYMBOL        FIFOPINPOLAR
  X:E604H         SYMBOL        FIFORESET
  B:00D0H.1       SYMBOL        FL
  X:E6CCH         SYMBOL        FLOWEDGE
  X:E6C8H         SYMBOL        FLOWEQ0CTL
  X:E6C9H         SYMBOL        FLOWEQ1CTL
  X:E6C7H         SYMBOL        FLOWLOGIC
  X:E6C6H         SYMBOL        FLOWSTATE
  X:E6CBH         SYMBOL        FLOWSTB
  X:E6CDH         SYMBOL        FLOWSTBHPERIOD
  X:E687H         SYMBOL        FNADDR
  X:E509H         SYMBOL        GPCR2
  X:E6F5H         SYMBOL        GPIFABORT
  X:E6C4H         SYMBOL        GPIFADRH
  X:E6C5H         SYMBOL        GPIFADRL
  X:E6C3H         SYMBOL        GPIFCTLCFG
  X:E60CH         SYMBOL        GPIFHOLDAMOUNT
  X:E6C1H         SYMBOL        GPIFIDLECS
  X:E6C2H         SYMBOL        GPIFIDLECTL
  X:E660H         SYMBOL        GPIFIE
  X:E661H         SYMBOL        GPIFIRQ
  X:E6F3H         SYMBOL        GPIFREADYCFG
  X:E6F4H         SYMBOL        GPIFREADYSTAT
  D:00BDH         SYMBOL        GPIFSGLDATH
  D:00BFH         SYMBOL        GPIFSGLDATLNOX
  D:00BEH         SYMBOL        GPIFSGLDATLX
  X:E6D1H         SYMBOL        GPIFTCB0
  X:E6D0H         SYMBOL        GPIFTCB1
  X:E6CFH         SYMBOL        GPIFTCB2
  X:E6CEH         SYMBOL        GPIFTCB3
  D:00BBH         SYMBOL        GPIFTRIG
  X:E6C0H         SYMBOL        GPIFWFSELECT
  X:E400H         SYMBOL        GPIF_WAVE_DATA
  X:E678H         SYMBOL        I2CS
  X:E67AH         SYMBOL        I2CTL
  X:E679H         SYMBOL        I2DAT
  X:E658H         SYMBOL        IBNIE
  X:E659H         SYMBOL        IBNIRQ
BL51 BANKED LINKER/LOCATER V6.02                                                      04/19/2018  15:18:09  PAGE 22


  D:00A8H         SYMBOL        IE
  B:0088H.1       SYMBOL        IE0
  B:0088H.3       SYMBOL        IE1
  X:E601H         SYMBOL        IFCONFIG
  X:E648H         SYMBOL        INPKTEND
  D:00A1H         SYMBOL        INT2CLR
  X:E666H         SYMBOL        INT2IVEC
  D:00A2H         SYMBOL        INT4CLR
  X:E667H         SYMBOL        INT4IVEC
  B:00D8H.3       SYMBOL        INT6
  X:E668H         SYMBOL        INTSETUP
  D:0080H         SYMBOL        IOA
  D:0090H         SYMBOL        IOB
  D:00A0H         SYMBOL        IOC
  D:00B0H         SYMBOL        IOD
  D:00B1H         SYMBOL        IOE
  D:00B8H         SYMBOL        IP
  B:0088H.0       SYMBOL        IT0
  B:0088H.2       SYMBOL        IT1
  X:E686H         SYMBOL        MICROFRAME
  D:0092H         SYMBOL        MPAGE
  X:E65AH         SYMBOL        NAKIE
  X:E65BH         SYMBOL        NAKIRQ
  D:00B2H         SYMBOL        OEA
  D:00B3H         SYMBOL        OEB
  D:00B4H         SYMBOL        OEC
  D:00B5H         SYMBOL        OED
  D:00B6H         SYMBOL        OEE
  X:E649H         SYMBOL        OUTPKTEND
  B:00D0H.2       SYMBOL        OV
  B:00D0H.0       SYMBOL        P
  B:0080H.0       SYMBOL        PA0
  B:0080H.1       SYMBOL        PA1
  B:0080H.2       SYMBOL        PA2
  B:0080H.3       SYMBOL        PA3
  B:0080H.4       SYMBOL        PA4
  B:0080H.5       SYMBOL        PA5
  B:0080H.6       SYMBOL        PA6
  B:0080H.7       SYMBOL        PA7
  B:0090H.0       SYMBOL        PB0
  B:0090H.1       SYMBOL        PB1
  B:0090H.2       SYMBOL        PB2
  B:0090H.3       SYMBOL        PB3
  B:0090H.4       SYMBOL        PB4
  B:0090H.5       SYMBOL        PB5
  B:0090H.6       SYMBOL        PB6
  B:0090H.7       SYMBOL        PB7
  B:00A0H.0       SYMBOL        PC0
  B:00A0H.1       SYMBOL        PC1
  B:00A0H.2       SYMBOL        PC2
  B:00A0H.3       SYMBOL        PC3
  B:00A0H.4       SYMBOL        PC4
  B:00A0H.5       SYMBOL        PC5
  B:00A0H.6       SYMBOL        PC6
  B:00A0H.7       SYMBOL        PC7
  D:0087H         SYMBOL        PCON
  B:00B0H.0       SYMBOL        PD0
BL51 BANKED LINKER/LOCATER V6.02                                                      04/19/2018  15:18:09  PAGE 23


  B:00B0H.1       SYMBOL        PD1
  B:00B0H.2       SYMBOL        PD2
  B:00B0H.3       SYMBOL        PD3
  B:00B0H.4       SYMBOL        PD4
  B:00B0H.5       SYMBOL        PD5
  B:00B0H.6       SYMBOL        PD6
  B:00B0H.7       SYMBOL        PD7
  B:00F8H.1       SYMBOL        PI2C
  X:E602H         SYMBOL        PINFLAGSAB
  X:E603H         SYMBOL        PINFLAGSCD
  X:E670H         SYMBOL        PORTACFG
  X:E671H         SYMBOL        PORTCCFG
  X:E672H         SYMBOL        PORTECFG
  B:00B8H.4       SYMBOL        PS0
  B:00B8H.6       SYMBOL        PS1
  D:00D0H         SYMBOL        PSW
  B:00B8H.1       SYMBOL        PT0
  B:00B8H.3       SYMBOL        PT1
  B:00B8H.5       SYMBOL        PT2
  B:00F8H.0       SYMBOL        PUSB
  B:00B8H.0       SYMBOL        PX0
  B:00B8H.2       SYMBOL        PX1
  B:0098H.2       SYMBOL        RB8
  B:00C0H.2       SYMBOL        RB81
  D:00CBH         SYMBOL        RCAP2H
  D:00CAH         SYMBOL        RCAP2L
  B:00C8H.5       SYMBOL        RCLK
  B:0098H.4       SYMBOL        REN
  B:00C0H.4       SYMBOL        REN1
  B:00D8H.4       SYMBOL        RESI
  X:E480H         SYMBOL        RES_WAVEDATA_END
  X:E60BH         SYMBOL        REVCTL
  X:E60AH         SYMBOL        REVID
  B:0098H.0       SYMBOL        RI
  B:00C0H.0       SYMBOL        RI1
  B:00D0H.3       SYMBOL        RS0
  B:00D0H.4       SYMBOL        RS1
  D:0099H         SYMBOL        SBUF0
  D:00C1H         SYMBOL        SBUF1
  D:0098H         SYMBOL        SCON0
  D:00C0H         SYMBOL        SCON1
  X:E6B8H         SYMBOL        SETUPDAT
  B:0098H.7       SYMBOL        SM0
  B:00C0H.7       SYMBOL        SM01
  B:0098H.6       SYMBOL        SM1
  B:00C0H.6       SYMBOL        SM11
  B:0098H.5       SYMBOL        SM2
  B:00C0H.5       SYMBOL        SM21
  B:00D8H.7       SYMBOL        SMOD1
  D:0081H         SYMBOL        SP
  X:E6B5H         SYMBOL        SUDPTRCTL
  X:E6B3H         SYMBOL        SUDPTRH
  X:E6B4H         SYMBOL        SUDPTRL
  N:0000H         SYMBOL        SUSP
  X:E681H         SYMBOL        SUSPEND
  D:00C8H         SYMBOL        T2CON
  B:0098H.3       SYMBOL        TB8
BL51 BANKED LINKER/LOCATER V6.02                                                      04/19/2018  15:18:09  PAGE 24


  B:00C0H.3       SYMBOL        TB81
  B:00C8H.4       SYMBOL        TCLK
  D:0088H         SYMBOL        TCON
  X:E6F9H         SYMBOL        TESTCFG
  B:0088H.5       SYMBOL        TF0
  B:0088H.7       SYMBOL        TF1
  B:00C8H.7       SYMBOL        TF2
  D:008CH         SYMBOL        TH0
  D:008DH         SYMBOL        TH1
  D:00CDH         SYMBOL        TH2
  B:0098H.1       SYMBOL        TI
  B:00C0H.1       SYMBOL        TI1
  D:008AH         SYMBOL        TL0
  D:008BH         SYMBOL        TL1
  D:00CCH         SYMBOL        TL2
  D:0089H         SYMBOL        TMOD
  X:E683H         SYMBOL        TOGCTL
  B:0088H.4       SYMBOL        TR0
  B:0088H.6       SYMBOL        TR1
  B:00C8H.2       SYMBOL        TR2
  X:E608H         SYMBOL        UART230
  X:E67DH         SYMBOL        UDMACRCH
  X:E67EH         SYMBOL        UDMACRCL
  X:E67FH         SYMBOL        UDMACRCQUAL
  X:E680H         SYMBOL        USBCS
  X:E662H         SYMBOL        USBERRIE
  X:E663H         SYMBOL        USBERRIRQ
  X:E684H         SYMBOL        USBFRAMEH
  X:E685H         SYMBOL        USBFRAMEL
  X:E65CH         SYMBOL        USBIE
  X:E65DH         SYMBOL        USBIRQ
  X:E6FAH         SYMBOL        USBTEST
  X:E682H         SYMBOL        WAKEUPCS
  X:E6F0H         SYMBOL        XGPIFSGLDATH
  X:E6F2H         SYMBOL        XGPIFSGLDATLNOX
  X:E6F1H         SYMBOL        XGPIFSGLDATLX
  C:0CD9H         LINE#         22
  C:0CDCH         LINE#         23
  C:0CDDH         LINE#         24
  C:0CDFH         LINE#         25
  C:0CE0H         LINE#         27
  C:0CE3H         LINE#         28
  C:0CE4H         LINE#         30
  C:0CE7H         LINE#         32
  C:0CE8H         LINE#         33
  C:0CE9H         LINE#         34
  C:0CEAH         LINE#         35
  C:0CEBH         LINE#         36
  C:0CECH         LINE#         37
  -------         ENDMOD        SUSP

  -------         MODULE        DELAY
  C:0000H         SYMBOL        _ICE_DUMMY_
  C:0AB2H         PUBLIC        _EZUSB_Delay
  -------         PROC          _EZUSB_DELAY
  D:0018H         SYMBOL        ms
  C:0AB2H         LINE#         39
BL51 BANKED LINKER/LOCATER V6.02                                                      04/19/2018  15:18:09  PAGE 25


  C:0AB6H         LINE#         40
  C:0AB6H         LINE#         46
  C:0ABEH         LINE#         47
  C:0AD0H         LINE#         48
  C:0ADAH         LINE#         49
  C:0AE5H         LINE#         51
  C:0AF2H         LINE#         52
  C:0AF7H         LINE#         53
  -------         ENDPROC       _EZUSB_DELAY
  -------         ENDMOD        DELAY

  -------         MODULE        DELAY1MS
  C:0CD9H         SEGMENT       EZUSB
  C:0CEDH         PUBLIC        EZUSB_DELAY1MS
  B:00D0H.6       SYMBOL        AC
  D:00E0H         SYMBOL        ACC
  D:009AH         SYMBOL        APTR1H
  D:009BH         SYMBOL        APTR1L
  D:009AH         SYMBOL        AUTOPTR1H
  D:009BH         SYMBOL        AUTOPTR1L
  D:009AH         SYMBOL        AUTOPTRH1
  D:009DH         SYMBOL        AUTOPTRH2
  D:009BH         SYMBOL        AUTOPTRL1
  D:009EH         SYMBOL        AUTOPTRL2
  D:00AFH         SYMBOL        AUTOPTRSETUP
  D:00F0H         SYMBOL        B
  X:E606H         SYMBOL        BPADDRH
  X:E607H         SYMBOL        BPADDRL
  X:E605H         SYMBOL        BREAKPT
  D:008EH         SYMBOL        CKCON
  X:E665H         SYMBOL        CLRERRCNT
  X:E600H         SYMBOL        CPUCS
  B:00C8H.0       SYMBOL        CP_RL2
  X:E6FBH         SYMBOL        CT1
  X:E6FCH         SYMBOL        CT2
  X:E6FDH         SYMBOL        CT3
  X:E6FEH         SYMBOL        CT4
  B:00D0H.7       SYMBOL        CY
  B:00C8H.1       SYMBOL        C_T2
  X:E6F8H         SYMBOL        DBUG
  N:0000H         SYMBOL        DELAY1MS
  D:0083H         SYMBOL        DPH
  D:0085H         SYMBOL        DPH1
  D:0082H         SYMBOL        DPL
  D:0084H         SYMBOL        DPL1
  D:0086H         SYMBOL        DPS
  B:00A8H.7       SYMBOL        EA
  X:E62AH         SYMBOL        ECC1B0
  X:E62BH         SYMBOL        ECC1B1
  X:E62CH         SYMBOL        ECC1B2
  X:E62DH         SYMBOL        ECC2B0
  X:E62EH         SYMBOL        ECC2B1
  X:E62FH         SYMBOL        ECC2B2
  X:E628H         SYMBOL        ECCCFG
  X:E629H         SYMBOL        ECCRESET
  B:00E8H.1       SYMBOL        EI2C
  D:00D8H         SYMBOL        EICON
BL51 BANKED LINKER/LOCATER V6.02                                                      04/19/2018  15:18:09  PAGE 26


  D:00E8H         SYMBOL        EIE
  B:00E8H.2       SYMBOL        EIEX4
  B:00E8H.3       SYMBOL        EIEX5
  B:00E8H.4       SYMBOL        EIEX6
  D:00F8H         SYMBOL        EIP
  B:00F8H.2       SYMBOL        EIPX4
  B:00F8H.3       SYMBOL        EIPX5
  B:00F8H.4       SYMBOL        EIPX6
  D:00BAH         SYMBOL        EP01STAT
  X:E68AH         SYMBOL        EP0BCH
  X:E68BH         SYMBOL        EP0BCL
  X:E740H         SYMBOL        EP0BUF
  X:E6A0H         SYMBOL        EP0CS
  X:E68FH         SYMBOL        EP1INBC
  X:E7C0H         SYMBOL        EP1INBUF
  X:E611H         SYMBOL        EP1INCFG
  X:E6A2H         SYMBOL        EP1INCS
  X:E68DH         SYMBOL        EP1OUTBC
  X:E780H         SYMBOL        EP1OUTBUF
  X:E610H         SYMBOL        EP1OUTCFG
  X:E6A1H         SYMBOL        EP1OUTCS
  D:00AAH         SYMBOL        EP2468STAT
  D:00ABH         SYMBOL        EP24FIFOFLGS
  X:E620H         SYMBOL        EP2AUTOINLENH
  X:E621H         SYMBOL        EP2AUTOINLENL
  X:E690H         SYMBOL        EP2BCH
  X:E691H         SYMBOL        EP2BCL
  X:E612H         SYMBOL        EP2CFG
  X:E6A3H         SYMBOL        EP2CS
  X:E6ABH         SYMBOL        EP2FIFOBCH
  X:E6ACH         SYMBOL        EP2FIFOBCL
  X:F000H         SYMBOL        EP2FIFOBUF
  X:E618H         SYMBOL        EP2FIFOCFG
  X:E6A7H         SYMBOL        EP2FIFOFLGS
  X:E650H         SYMBOL        EP2FIFOIE
  X:E651H         SYMBOL        EP2FIFOIRQ
  X:E630H         SYMBOL        EP2FIFOPFH
  X:E631H         SYMBOL        EP2FIFOPFL
  X:E6D2H         SYMBOL        EP2GPIFFLGSEL
  X:E6D3H         SYMBOL        EP2GPIFPFSTOP
  X:E6D0H         SYMBOL        EP2GPIFTCH
  X:E6D1H         SYMBOL        EP2GPIFTCL
  X:E6D4H         SYMBOL        EP2GPIFTRIG
  X:E640H         SYMBOL        EP2ISOINPKTS
  X:E622H         SYMBOL        EP4AUTOINLENH
  X:E623H         SYMBOL        EP4AUTOINLENL
  X:E694H         SYMBOL        EP4BCH
  X:E695H         SYMBOL        EP4BCL
  X:E613H         SYMBOL        EP4CFG
  X:E6A4H         SYMBOL        EP4CS
  X:E6ADH         SYMBOL        EP4FIFOBCH
  X:E6AEH         SYMBOL        EP4FIFOBCL
  X:F400H         SYMBOL        EP4FIFOBUF
  X:E619H         SYMBOL        EP4FIFOCFG
  X:E6A8H         SYMBOL        EP4FIFOFLGS
  X:E652H         SYMBOL        EP4FIFOIE
  X:E653H         SYMBOL        EP4FIFOIRQ
BL51 BANKED LINKER/LOCATER V6.02                                                      04/19/2018  15:18:09  PAGE 27


  X:E632H         SYMBOL        EP4FIFOPFH
  X:E633H         SYMBOL        EP4FIFOPFL
  X:E6DAH         SYMBOL        EP4GPIFFLGSEL
  X:E6DBH         SYMBOL        EP4GPIFPFSTOP
  X:E6D0H         SYMBOL        EP4GPIFTCH
  X:E6D1H         SYMBOL        EP4GPIFTCL
  X:E6DCH         SYMBOL        EP4GPIFTRIG
  X:E641H         SYMBOL        EP4ISOINPKTS
  D:00ACH         SYMBOL        EP68FIFOFLGS
  X:E624H         SYMBOL        EP6AUTOINLENH
  X:E625H         SYMBOL        EP6AUTOINLENL
  X:E698H         SYMBOL        EP6BCH
  X:E699H         SYMBOL        EP6BCL
  X:E614H         SYMBOL        EP6CFG
  X:E6A5H         SYMBOL        EP6CS
  X:E6AFH         SYMBOL        EP6FIFOBCH
  X:E6B0H         SYMBOL        EP6FIFOBCL
  X:F800H         SYMBOL        EP6FIFOBUF
  X:E61AH         SYMBOL        EP6FIFOCFG
  X:E6A9H         SYMBOL        EP6FIFOFLGS
  X:E654H         SYMBOL        EP6FIFOIE
  X:E655H         SYMBOL        EP6FIFOIRQ
  X:E634H         SYMBOL        EP6FIFOPFH
  X:E635H         SYMBOL        EP6FIFOPFL
  X:E6E2H         SYMBOL        EP6GPIFFLGSEL
  X:E6E3H         SYMBOL        EP6GPIFPFSTOP
  X:E6D0H         SYMBOL        EP6GPIFTCH
  X:E6D1H         SYMBOL        EP6GPIFTCL
  X:E6E4H         SYMBOL        EP6GPIFTRIG
  X:E642H         SYMBOL        EP6ISOINPKTS
  X:E626H         SYMBOL        EP8AUTOINLENH
  X:E627H         SYMBOL        EP8AUTOINLENL
  X:E69CH         SYMBOL        EP8BCH
  X:E69DH         SYMBOL        EP8BCL
  X:E615H         SYMBOL        EP8CFG
  X:E6A6H         SYMBOL        EP8CS
  X:E6B1H         SYMBOL        EP8FIFOBCH
  X:E6B2H         SYMBOL        EP8FIFOBCL
  X:FC00H         SYMBOL        EP8FIFOBUF
  X:E61BH         SYMBOL        EP8FIFOCFG
  X:E6AAH         SYMBOL        EP8FIFOFLGS
  X:E656H         SYMBOL        EP8FIFOIE
  X:E657H         SYMBOL        EP8FIFOIRQ
  X:E636H         SYMBOL        EP8FIFOPFH
  X:E637H         SYMBOL        EP8FIFOPFL
  X:E6EAH         SYMBOL        EP8GPIFFLGSEL
  X:E6EBH         SYMBOL        EP8GPIFPFSTOP
  X:E6D0H         SYMBOL        EP8GPIFTCH
  X:E6D1H         SYMBOL        EP8GPIFTCL
  X:E6ECH         SYMBOL        EP8GPIFTRIG
  X:E643H         SYMBOL        EP8ISOINPKTS
  X:E65EH         SYMBOL        EPIE
  X:E65FH         SYMBOL        EPIRQ
  B:00D8H.5       SYMBOL        ERESI
  X:E664H         SYMBOL        ERRCNTLIM
  C:0CFDH         SYMBOL        ER_END
  B:00A8H.4       SYMBOL        ES0
BL51 BANKED LINKER/LOCATER V6.02                                                      04/19/2018  15:18:09  PAGE 28


  B:00A8H.6       SYMBOL        ES1
  B:00A8H.1       SYMBOL        ET0
  B:00A8H.3       SYMBOL        ET1
  B:00A8H.5       SYMBOL        ET2
  B:00E8H.0       SYMBOL        EUSB
  B:00A8H.0       SYMBOL        EX0
  B:00A8H.2       SYMBOL        EX1
  B:00C8H.3       SYMBOL        EXEN2
  B:00C8H.6       SYMBOL        EXF2
  D:0091H         SYMBOL        EXIF
  X:E67BH         SYMBOL        EXTAUTODAT1
  X:E67CH         SYMBOL        EXTAUTODAT2
  B:00D0H.5       SYMBOL        F0
  X:E609H         SYMBOL        FIFOPINPOLAR
  X:E604H         SYMBOL        FIFORESET
  B:00D0H.1       SYMBOL        FL
  X:E6CCH         SYMBOL        FLOWEDGE
  X:E6C8H         SYMBOL        FLOWEQ0CTL
  X:E6C9H         SYMBOL        FLOWEQ1CTL
  X:E6C7H         SYMBOL        FLOWLOGIC
  X:E6C6H         SYMBOL        FLOWSTATE
  X:E6CBH         SYMBOL        FLOWSTB
  X:E6CDH         SYMBOL        FLOWSTBHPERIOD
  X:E687H         SYMBOL        FNADDR
  X:E509H         SYMBOL        GPCR2
  X:E6F5H         SYMBOL        GPIFABORT
  X:E6C4H         SYMBOL        GPIFADRH
  X:E6C5H         SYMBOL        GPIFADRL
  X:E6C3H         SYMBOL        GPIFCTLCFG
  X:E60CH         SYMBOL        GPIFHOLDAMOUNT
  X:E6C1H         SYMBOL        GPIFIDLECS
  X:E6C2H         SYMBOL        GPIFIDLECTL
  X:E660H         SYMBOL        GPIFIE
  X:E661H         SYMBOL        GPIFIRQ
  X:E6F3H         SYMBOL        GPIFREADYCFG
  X:E6F4H         SYMBOL        GPIFREADYSTAT
  D:00BDH         SYMBOL        GPIFSGLDATH
  D:00BFH         SYMBOL        GPIFSGLDATLNOX
  D:00BEH         SYMBOL        GPIFSGLDATLX
  X:E6D1H         SYMBOL        GPIFTCB0
  X:E6D0H         SYMBOL        GPIFTCB1
  X:E6CFH         SYMBOL        GPIFTCB2
  X:E6CEH         SYMBOL        GPIFTCB3
  D:00BBH         SYMBOL        GPIFTRIG
  X:E6C0H         SYMBOL        GPIFWFSELECT
  X:E400H         SYMBOL        GPIF_WAVE_DATA
  X:E678H         SYMBOL        I2CS
  X:E67AH         SYMBOL        I2CTL
  X:E679H         SYMBOL        I2DAT
  X:E658H         SYMBOL        IBNIE
  X:E659H         SYMBOL        IBNIRQ
  D:00A8H         SYMBOL        IE
  B:0088H.1       SYMBOL        IE0
  B:0088H.3       SYMBOL        IE1
  X:E601H         SYMBOL        IFCONFIG
  X:E648H         SYMBOL        INPKTEND
  D:00A1H         SYMBOL        INT2CLR
BL51 BANKED LINKER/LOCATER V6.02                                                      04/19/2018  15:18:09  PAGE 29


  X:E666H         SYMBOL        INT2IVEC
  D:00A2H         SYMBOL        INT4CLR
  X:E667H         SYMBOL        INT4IVEC
  B:00D8H.3       SYMBOL        INT6
  X:E668H         SYMBOL        INTSETUP
  D:0080H         SYMBOL        IOA
  D:0090H         SYMBOL        IOB
  D:00A0H         SYMBOL        IOC
  D:00B0H         SYMBOL        IOD
  D:00B1H         SYMBOL        IOE
  D:00B8H         SYMBOL        IP
  B:0088H.0       SYMBOL        IT0
  B:0088H.2       SYMBOL        IT1
  C:0CF6H         SYMBOL        LOOP
  X:E686H         SYMBOL        MICROFRAME
  D:0092H         SYMBOL        MPAGE
  X:E65AH         SYMBOL        NAKIE
  X:E65BH         SYMBOL        NAKIRQ
  D:00B2H         SYMBOL        OEA
  D:00B3H         SYMBOL        OEB
  D:00B4H         SYMBOL        OEC
  D:00B5H         SYMBOL        OED
  D:00B6H         SYMBOL        OEE
  X:E649H         SYMBOL        OUTPKTEND
  B:00D0H.2       SYMBOL        OV
  B:00D0H.0       SYMBOL        P
  B:0080H.0       SYMBOL        PA0
  B:0080H.1       SYMBOL        PA1
  B:0080H.2       SYMBOL        PA2
  B:0080H.3       SYMBOL        PA3
  B:0080H.4       SYMBOL        PA4
  B:0080H.5       SYMBOL        PA5
  B:0080H.6       SYMBOL        PA6
  B:0080H.7       SYMBOL        PA7
  B:0090H.0       SYMBOL        PB0
  B:0090H.1       SYMBOL        PB1
  B:0090H.2       SYMBOL        PB2
  B:0090H.3       SYMBOL        PB3
  B:0090H.4       SYMBOL        PB4
  B:0090H.5       SYMBOL        PB5
  B:0090H.6       SYMBOL        PB6
  B:0090H.7       SYMBOL        PB7
  B:00A0H.0       SYMBOL        PC0
  B:00A0H.1       SYMBOL        PC1
  B:00A0H.2       SYMBOL        PC2
  B:00A0H.3       SYMBOL        PC3
  B:00A0H.4       SYMBOL        PC4
  B:00A0H.5       SYMBOL        PC5
  B:00A0H.6       SYMBOL        PC6
  B:00A0H.7       SYMBOL        PC7
  D:0087H         SYMBOL        PCON
  B:00B0H.0       SYMBOL        PD0
  B:00B0H.1       SYMBOL        PD1
  B:00B0H.2       SYMBOL        PD2
  B:00B0H.3       SYMBOL        PD3
  B:00B0H.4       SYMBOL        PD4
  B:00B0H.5       SYMBOL        PD5
BL51 BANKED LINKER/LOCATER V6.02                                                      04/19/2018  15:18:09  PAGE 30


  B:00B0H.6       SYMBOL        PD6
  B:00B0H.7       SYMBOL        PD7
  B:00F8H.1       SYMBOL        PI2C
  X:E602H         SYMBOL        PINFLAGSAB
  X:E603H         SYMBOL        PINFLAGSCD
  X:E670H         SYMBOL        PORTACFG
  X:E671H         SYMBOL        PORTCCFG
  X:E672H         SYMBOL        PORTECFG
  B:00B8H.4       SYMBOL        PS0
  B:00B8H.6       SYMBOL        PS1
  D:00D0H         SYMBOL        PSW
  B:00B8H.1       SYMBOL        PT0
  B:00B8H.3       SYMBOL        PT1
  B:00B8H.5       SYMBOL        PT2
  B:00F8H.0       SYMBOL        PUSB
  B:00B8H.0       SYMBOL        PX0
  B:00B8H.2       SYMBOL        PX1
  B:0098H.2       SYMBOL        RB8
  B:00C0H.2       SYMBOL        RB81
  D:00CBH         SYMBOL        RCAP2H
  D:00CAH         SYMBOL        RCAP2L
  B:00C8H.5       SYMBOL        RCLK
  B:0098H.4       SYMBOL        REN
  B:00C0H.4       SYMBOL        REN1
  B:00D8H.4       SYMBOL        RESI
  X:E480H         SYMBOL        RES_WAVEDATA_END
  X:E60BH         SYMBOL        REVCTL
  X:E60AH         SYMBOL        REVID
  B:0098H.0       SYMBOL        RI
  B:00C0H.0       SYMBOL        RI1
  B:00D0H.3       SYMBOL        RS0
  B:00D0H.4       SYMBOL        RS1
  D:0099H         SYMBOL        SBUF0
  D:00C1H         SYMBOL        SBUF1
  D:0098H         SYMBOL        SCON0
  D:00C0H         SYMBOL        SCON1
  X:E6B8H         SYMBOL        SETUPDAT
  B:0098H.7       SYMBOL        SM0
  B:00C0H.7       SYMBOL        SM01
  B:0098H.6       SYMBOL        SM1
  B:00C0H.6       SYMBOL        SM11
  B:0098H.5       SYMBOL        SM2
  B:00C0H.5       SYMBOL        SM21
  B:00D8H.7       SYMBOL        SMOD1
  D:0081H         SYMBOL        SP
  X:E6B5H         SYMBOL        SUDPTRCTL
  X:E6B3H         SYMBOL        SUDPTRH
  X:E6B4H         SYMBOL        SUDPTRL
  X:E681H         SYMBOL        SUSPEND
  D:00C8H         SYMBOL        T2CON
  B:0098H.3       SYMBOL        TB8
  B:00C0H.3       SYMBOL        TB81
  B:00C8H.4       SYMBOL        TCLK
  D:0088H         SYMBOL        TCON
  X:E6F9H         SYMBOL        TESTCFG
  B:0088H.5       SYMBOL        TF0
  B:0088H.7       SYMBOL        TF1
BL51 BANKED LINKER/LOCATER V6.02                                                      04/19/2018  15:18:09  PAGE 31


  B:00C8H.7       SYMBOL        TF2
  D:008CH         SYMBOL        TH0
  D:008DH         SYMBOL        TH1
  D:00CDH         SYMBOL        TH2
  B:0098H.1       SYMBOL        TI
  B:00C0H.1       SYMBOL        TI1
  D:008AH         SYMBOL        TL0
  D:008BH         SYMBOL        TL1
  D:00CCH         SYMBOL        TL2
  D:0089H         SYMBOL        TMOD
  X:E683H         SYMBOL        TOGCTL
  B:0088H.4       SYMBOL        TR0
  B:0088H.6       SYMBOL        TR1
  B:00C8H.2       SYMBOL        TR2
  X:E608H         SYMBOL        UART230
  X:E67DH         SYMBOL        UDMACRCH
  X:E67EH         SYMBOL        UDMACRCL
  X:E67FH         SYMBOL        UDMACRCQUAL
  X:E680H         SYMBOL        USBCS
  X:E662H         SYMBOL        USBERRIE
  X:E663H         SYMBOL        USBERRIRQ
  X:E684H         SYMBOL        USBFRAMEH
  X:E685H         SYMBOL        USBFRAMEL
  X:E65CH         SYMBOL        USBIE
  X:E65DH         SYMBOL        USBIRQ
  X:E6FAH         SYMBOL        USBTEST
  X:E682H         SYMBOL        WAKEUPCS
  X:E6F0H         SYMBOL        XGPIFSGLDATH
  X:E6F2H         SYMBOL        XGPIFSGLDATLNOX
  X:E6F1H         SYMBOL        XGPIFSGLDATLX
  C:0CEDH         LINE#         48
  C:0CEFH         LINE#         49
  C:0CF1H         LINE#         50
  C:0CF4H         LINE#         51
  C:0CF6H         LINE#         53
  C:0CF7H         LINE#         54
  C:0CF9H         LINE#         55
  C:0CFBH         LINE#         56
  C:0CFDH         LINE#         58
  -------         ENDMOD        DELAY1MS

  -------         MODULE        USBJMPTBL
  C:0B00H         SEGMENT       ?PR?USB_JUMP_TABLE?USBJT
  N:0045H         PUBLIC        USB_INT2AUTOVECTOR
  N:0055H         PUBLIC        USB_INT4AUTOVECTOR
  C:0B00H         PUBLIC        USB_JUMP_TABLE
  N:0000H         SYMBOL        USBJMPTBL
  C:0043H         LINE#         49
  C:0053H         LINE#         53
  C:0B00H         LINE#         61
  C:0B04H         LINE#         63
  C:0B08H         LINE#         65
  C:0B0CH         LINE#         67
  C:0B10H         LINE#         69
  C:0B14H         LINE#         71
  C:0B18H         LINE#         73
  C:0B1CH         LINE#         75
BL51 BANKED LINKER/LOCATER V6.02                                                      04/19/2018  15:18:09  PAGE 32


  C:0B20H         LINE#         77
  C:0B24H         LINE#         79
  C:0B28H         LINE#         81
  C:0B2CH         LINE#         83
  C:0B30H         LINE#         85
  C:0B34H         LINE#         87
  C:0B38H         LINE#         89
  C:0B3CH         LINE#         91
  C:0B40H         LINE#         93
  C:0B44H         LINE#         95
  C:0B48H         LINE#         97
  C:0B4CH         LINE#         99
  C:0B50H         LINE#         101
  C:0B54H         LINE#         103
  C:0B58H         LINE#         105
  C:0B5CH         LINE#         107
  C:0B60H         LINE#         109
  C:0B64H         LINE#         111
  C:0B68H         LINE#         113
  C:0B6CH         LINE#         115
  C:0B70H         LINE#         117
  C:0B74H         LINE#         119
  C:0B78H         LINE#         121
  C:0B7CH         LINE#         123
  C:0B80H         LINE#         126
  C:0B84H         LINE#         128
  C:0B88H         LINE#         130
  C:0B8CH         LINE#         132
  C:0B90H         LINE#         134
  C:0B94H         LINE#         136
  C:0B98H         LINE#         138
  C:0B9CH         LINE#         140
  C:0BA0H         LINE#         142
  C:0BA4H         LINE#         144
  C:0BA8H         LINE#         146
  C:0BACH         LINE#         148
  C:0BB0H         LINE#         150
  C:0BB4H         LINE#         152
  -------         ENDMOD        USBJMPTBL

  -------         MODULE        INTERRUPCIONES
  C:0000H         SYMBOL        _ICE_DUMMY_
  D:008CH         PUBLIC        TH0
  D:008DH         PUBLIC        TH1
  D:008AH         PUBLIC        TL0
  D:008BH         PUBLIC        TL1
  C:0F2FH         PUBLIC        timer0
  C:0DF2H         PUBLIC        timer1
  B:0088H.4       PUBLIC        TR0
  B:0088H.6       PUBLIC        TR1
  -------         PROC          TIMER0
  C:0F2FH         LINE#         10
  C:0F33H         LINE#         14
  C:0F35H         LINE#         15
  C:0F3BH         LINE#         16
  C:0F41H         LINE#         17
  C:0F43H         LINE#         20
BL51 BANKED LINKER/LOCATER V6.02                                                      04/19/2018  15:18:09  PAGE 33


  C:0F4BH         LINE#         21
  -------         ENDPROC       TIMER0
  -------         PROC          TIMER1
  C:0DF2H         LINE#         29
  C:0DF6H         LINE#         33
  C:0DF8H         LINE#         34
  C:0DFEH         LINE#         35
  C:0E04H         LINE#         36
  C:0E06H         LINE#         39
  C:0E0EH         LINE#         40
  C:0E16H         LINE#         41
  C:0E1EH         LINE#         42
  C:0E26H         LINE#         43
  -------         ENDPROC       TIMER1
  -------         ENDMOD        INTERRUPCIONES

  -------         MODULE        PEDALERA
  C:0000H         SYMBOL        _ICE_DUMMY_
  C:1093H         PUBLIC        ISR_Errorlimit
  B:00A8H.7       PUBLIC        EA
  C:0AF8H         PUBLIC        DR_SetConfiguration
  B:0090H.2       PUBLIC        AUXIN
  D:0021H         PUBLIC        AlternateSetting
  D:0022H         PUBLIC        timer1_tiempo_on_disparo_retrasado
  C:1084H         PUBLIC        ISR_Ep0in
  C:1086H         PUBLIC        ISR_Ep1in
  C:100BH         PUBLIC        TD_Init
  C:1085H         PUBLIC        ISR_Ep0out
  C:1087H         PUBLIC        ISR_Ep1out
  C:0080H         PUBLIC        TD_Poll
  B:00B0H.1       PUBLIC        VSYNC
  C:10A4H         PUBLIC        ISR_GpifComplete
  D:0024H         PUBLIC        test_disparo
  D:0025H         PUBLIC        packetSize
  B:0090H.5       PUBLIC        PORTB_5
  B:0090H.6       PUBLIC        PORTB_6
  B:0090H.0       PUBLIC        CINE
  D:0027H         PUBLIC        timer1_delay_disparo
  C:107CH         PUBLIC        DR_GetStatus
  C:108DH         PUBLIC        ISR_Ep0pingnak
  B:0020H.4       PUBLIC        in_enable
  C:108EH         PUBLIC        ISR_Ep1pingnak
  C:10A5H         PUBLIC        ISR_GpifWaveform
  C:1094H         PUBLIC        ISR_Ep2piderror
  C:108FH         PUBLIC        ISR_Ep2pingnak
  D:0029H         PUBLIC        estado_salida_pulsada
  C:1095H         PUBLIC        ISR_Ep4piderror
  C:1090H         PUBLIC        ISR_Ep4pingnak
  C:1096H         PUBLIC        ISR_Ep6piderror
  C:1091H         PUBLIC        ISR_Ep6pingnak
  C:1097H         PUBLIC        ISR_Ep8piderror
  C:1092H         PUBLIC        ISR_Ep8pingnak
  D:002AH         PUBLIC        disparo_por_cine
  D:002BH         PUBLIC        delta_tick_1
  B:00B0H.2       PUBLIC        RELE_AUX3
  D:0091H         PUBLIC        EXIF
  C:102FH         PUBLIC        DR_GetInterface
BL51 BANKED LINKER/LOCATER V6.02                                                      04/19/2018  15:18:09  PAGE 34


  C:107EH         PUBLIC        DR_ClearFeature
  D:0089H         PUBLIC        TMOD
  C:0A13H         PUBLIC        _AntiRebotePedales
  C:109CH         PUBLIC        ISR_Ep2eflag
  C:10A0H         PUBLIC        ISR_Ep2fflag
  C:109DH         PUBLIC        ISR_Ep4eflag
  C:1064H         PUBLIC        DR_SetInterface
  C:10A1H         PUBLIC        ISR_Ep4fflag
  C:109EH         PUBLIC        ISR_Ep6eflag
  C:10A2H         PUBLIC        ISR_Ep6fflag
  C:107AH         PUBLIC        DR_GetDescriptor
  C:109FH         PUBLIC        ISR_Ep8eflag
  C:10A3H         PUBLIC        ISR_Ep8fflag
  B:0090H.1       PUBLIC        SCOPIA
  B:00B0H.3       PUBLIC        RELE_IRIS
  C:1098H         PUBLIC        ISR_Ep2pflag
  C:1099H         PUBLIC        ISR_Ep4pflag
  D:002DH         PUBLIC        estado_pedales
  C:109AH         PUBLIC        ISR_Ep6pflag
  B:00A8H.1       PUBLIC        ET0
  B:00A8H.3       PUBLIC        ET1
  C:109BH         PUBLIC        ISR_Ep8pflag
  D:0030H         PUBLIC        estado_disparo_latch
  D:008CH         PUBLIC        TH0
  D:008DH         PUBLIC        TH1
  D:0031H         PUBLIC        modo_auto_gain
  D:008AH         PUBLIC        TL0
  D:008BH         PUBLIC        TL1
  B:00B8H.1       PUBLIC        PT0
  C:0F92H         PUBLIC        ISR_Sudav
  B:00B8H.3       PUBLIC        PT1
  D:00B2H         PUBLIC        OEA
  D:00B3H         PUBLIC        OEB
  B:0088H.4       PUBLIC        TR0
  B:0088H.6       PUBLIC        TR1
  D:00B5H         PUBLIC        OED
  D:0090H         PUBLIC        IOB
  D:0032H         PUBLIC        tiempo_ref_fps
  D:00B0H         PUBLIC        IOD
  D:0034H         PUBLIC        timer1_tiempo_on_disparo
  C:0CFEH         PUBLIC        TD_Suspend
  D:0036H         PUBLIC        Configuration
  D:0037H         PUBLIC        timer0_tick
  D:0039H         PUBLIC        origen_pulso_entrada
  D:003AH         PUBLIC        timer1_tick
  C:1082H         PUBLIC        ISR_Ep0ack
  C:0D72H         PUBLIC        ISR_Highspeed
  C:0FC9H         PUBLIC        ISR_Sutok
  B:00B0H.6       PUBLIC        AUXOUT
  C:108CH         PUBLIC        ISR_Ibn
  B:0090H.3       PUBLIC        TRIGGER_EXT
  C:1088H         PUBLIC        ISR_Ep2inout
  C:0F50H         PUBLIC        timer0_init
  C:1089H         PUBLIC        ISR_Ep4inout
  C:0F71H         PUBLIC        timer1_init
  C:0396H         PUBLIC        DR_VendorCmnd
  C:1078H         PUBLIC        TD_Resume
BL51 BANKED LINKER/LOCATER V6.02                                                      04/19/2018  15:18:09  PAGE 35


  C:108AH         PUBLIC        ISR_Ep6inout
  C:0EE8H         PUBLIC        InicializarPuertos
  C:1083H         PUBLIC        ISR_Stub
  D:008EH         PUBLIC        CKCON
  C:108BH         PUBLIC        ISR_Ep8inout
  C:0C96H         PUBLIC        ISR_Ures
  B:00B0H.5       PUBLIC        TRIGGER_OUT
  B:00B0H.0       PUBLIC        CAMPO
  D:003CH         PUBLIC        tiempo_on_salida_pulsada
  B:00B0H.4       PUBLIC        RELE_HCINE
  D:003EH         PUBLIC        disparo_por_escopia
  C:1080H         PUBLIC        DR_SetFeature
  B:00B0H.7       PUBLIC        READY
  C:0FDFH         PUBLIC        ISR_Sof
  C:101DH         PUBLIC        DR_GetConfiguration
  C:0FB1H         PUBLIC        ISR_Susp
  B:0090H.4       PUBLIC        GRABMEM
  -------         PROC          TD_INIT
  C:100BH         LINE#         170
  C:100BH         LINE#         171
  C:100BH         LINE#         173
  C:1014H         LINE#         175
  C:1017H         LINE#         177
  C:101AH         LINE#         178
  -------         ENDPROC       TD_INIT
  -------         PROC          TD_POLL
  C:0080H         LINE#         181
  C:0080H         LINE#         182
  C:0080H         LINE#         184
  C:008BH         LINE#         185
  C:008BH         LINE#         186
  C:0090H         LINE#         187
  C:0095H         LINE#         188
  C:009AH         LINE#         190
  C:009FH         LINE#         191
  C:009FH         LINE#         194
  C:00A8H         LINE#         195
  C:00A8H         LINE#         197
  C:00C3H         LINE#         198
  C:00C3H         LINE#         199
  C:00C3H         LINE#         200
  C:00C3H         LINE#         201
  C:00DCH         LINE#         202
  C:00DCH         LINE#         203
  C:00DCH         LINE#         204
  C:00DCH         LINE#         205
  C:00E2H         LINE#         206
  C:00E2H         LINE#         207
  C:00E2H         LINE#         208
  C:00E2H         LINE#         209
  C:00E2H         LINE#         210
  C:00E2H         LINE#         211
  C:00E2H         LINE#         213
  C:00E4H         LINE#         214
  C:00E4H         LINE#         216
  C:00E4H         LINE#         217
  C:00E4H         LINE#         218
BL51 BANKED LINKER/LOCATER V6.02                                                      04/19/2018  15:18:09  PAGE 36


  C:00F9H         LINE#         221
  C:00F9H         LINE#         222
  C:00F9H         LINE#         223
  C:00F9H         LINE#         224
  C:00F9H         LINE#         225
  C:00F9H         LINE#         226
  C:00F9H         LINE#         227
  C:00F9H         LINE#         229
  C:00FBH         LINE#         230
  C:00FBH         LINE#         232
  C:00FBH         LINE#         233
  C:00FBH         LINE#         234
  C:0110H         LINE#         236
  C:0110H         LINE#         237
  C:0115H         LINE#         238
  C:0119H         LINE#         239
  C:011DH         LINE#         240
  C:011FH         LINE#         241
  C:011FH         LINE#         242
  C:011FH         LINE#         244
  C:0121H         LINE#         245
  C:0121H         LINE#         247
  C:0121H         LINE#         248
  C:0121H         LINE#         249
  C:013AH         LINE#         250
  C:013AH         LINE#         251
  C:0148H         LINE#         252
  C:0148H         LINE#         253
  C:014DH         LINE#         254
  C:0151H         LINE#         255
  C:0155H         LINE#         256
  C:0158H         LINE#         257
  C:015AH         LINE#         258
  C:015AH         LINE#         259
  C:015AH         LINE#         261
  C:015BH         LINE#         262
  C:015BH         LINE#         264
  C:015BH         LINE#         265
  C:015BH         LINE#         266
  C:0161H         LINE#         267
  C:0161H         LINE#         268
  C:0166H         LINE#         269
  C:016AH         LINE#         270
  C:016EH         LINE#         273
  C:0171H         LINE#         274
  C:0171H         LINE#         276
  C:0172H         LINE#         277
  C:0172H         LINE#         278
  C:0172H         LINE#         280
  C:0172H         LINE#         281
  C:0172H         LINE#         283
  C:0172H         LINE#         284
  C:0172H         LINE#         285
  C:0180H         LINE#         286
  C:0180H         LINE#         287
  C:0180H         LINE#         288
  C:0180H         LINE#         290
BL51 BANKED LINKER/LOCATER V6.02                                                      04/19/2018  15:18:09  PAGE 37


  C:018BH         LINE#         291
  C:018BH         LINE#         292
  C:018EH         LINE#         293
  C:0190H         LINE#         296
  C:0195H         LINE#         297
  C:0195H         LINE#         301
  C:01A3H         LINE#         302
  C:01A5H         LINE#         305
  C:01A6H         LINE#         306
  C:01A6H         LINE#         308
  C:01A6H         LINE#         309
  C:01A6H         LINE#         310
  C:01B4H         LINE#         311
  C:01B4H         LINE#         312
  C:01B7H         LINE#         313
  C:01BBH         LINE#         314
  C:01BEH         LINE#         315
  C:01C0H         LINE#         316
  C:01C0H         LINE#         317
  C:01C1H         LINE#         318
  C:01C1H         LINE#         320
  C:01C1H         LINE#         321
  C:01C1H         LINE#         323
  C:01CCH         LINE#         324
  C:01CCH         LINE#         325
  C:01CEH         LINE#         326
  C:01D3H         LINE#         327
  C:01D5H         LINE#         328
  C:01D8H         LINE#         329
  C:01D8H         LINE#         333
  C:01E6H         LINE#         334
  C:01E8H         LINE#         337
  C:01E9H         LINE#         338
  C:01E9H         LINE#         340
  C:01E9H         LINE#         341
  C:01E9H         LINE#         343
  C:01F4H         LINE#         344
  C:01F4H         LINE#         345
  C:01F6H         LINE#         347
  C:01FBH         LINE#         348
  C:01FDH         LINE#         349
  C:0200H         LINE#         350
  C:0200H         LINE#         354
  C:020EH         LINE#         355
  C:0210H         LINE#         358
  C:0211H         LINE#         359
  C:0211H         LINE#         360
  C:0211H         LINE#         362
  C:0211H         LINE#         363
  C:0211H         LINE#         365
  C:0211H         LINE#         366
  C:0211H         LINE#         367
  C:0222H         LINE#         368
  C:0222H         LINE#         369
  C:0222H         LINE#         370
  C:0222H         LINE#         372
  C:022DH         LINE#         373
BL51 BANKED LINKER/LOCATER V6.02                                                      04/19/2018  15:18:09  PAGE 38


  C:022DH         LINE#         374
  C:022FH         LINE#         375
  C:0232H         LINE#         377
  C:0234H         LINE#         378
  C:0234H         LINE#         382
  C:0242H         LINE#         383
  C:0244H         LINE#         385
  C:0245H         LINE#         386
  C:0245H         LINE#         388
  C:0245H         LINE#         389
  C:0245H         LINE#         390
  C:025AH         LINE#         391
  C:025AH         LINE#         392
  C:025DH         LINE#         393
  C:025FH         LINE#         394
  C:0262H         LINE#         395
  C:0262H         LINE#         396
  C:0263H         LINE#         397
  C:0263H         LINE#         399
  C:0263H         LINE#         400
  C:0263H         LINE#         401
  C:0275H         LINE#         402
  C:0278H         LINE#         405
  C:0283H         LINE#         406
  C:0283H         LINE#         407
  C:0285H         LINE#         408
  C:0287H         LINE#         409
  C:028AH         LINE#         410
  C:028AH         LINE#         414
  C:0298H         LINE#         415
  C:029AH         LINE#         418
  C:029BH         LINE#         419
  C:029BH         LINE#         421
  C:029BH         LINE#         422
  C:029BH         LINE#         423
  C:02ADH         LINE#         424
  C:02B0H         LINE#         427
  C:02BBH         LINE#         428
  C:02BBH         LINE#         429
  C:02BDH         LINE#         430
  C:02BFH         LINE#         431
  C:02C2H         LINE#         432
  C:02C2H         LINE#         436
  C:02D0H         LINE#         437
  C:02D2H         LINE#         440
  C:02D3H         LINE#         441
  C:02D3H         LINE#         442
  C:02D3H         LINE#         444
  C:02D3H         LINE#         445
  C:02D3H         LINE#         447
  C:02D3H         LINE#         448
  C:02D3H         LINE#         449
  C:02EFH         LINE#         450
  C:02EFH         LINE#         451
  C:02EFH         LINE#         452
  C:02EFH         LINE#         453
  C:02F5H         LINE#         454
BL51 BANKED LINKER/LOCATER V6.02                                                      04/19/2018  15:18:09  PAGE 39


  C:02F5H         LINE#         456
  C:02F8H         LINE#         457
  C:02F8H         LINE#         459
  C:02F8H         LINE#         460
  C:02F8H         LINE#         461
  C:030AH         LINE#         462
  C:030DH         LINE#         464
  C:0331H         LINE#         466
  C:0331H         LINE#         467
  C:0331H         LINE#         468
  C:0331H         LINE#         469
  C:0331H         LINE#         471
  C:0333H         LINE#         472
  C:0333H         LINE#         474
  C:0333H         LINE#         475
  C:0333H         LINE#         476
  C:0345H         LINE#         477
  C:0348H         LINE#         479
  C:0369H         LINE#         480
  C:0369H         LINE#         481
  C:036AH         LINE#         482
  C:036AH         LINE#         483
  C:036CH         LINE#         485
  C:036FH         LINE#         487
  C:0370H         LINE#         488
  C:0370H         LINE#         490
  C:0370H         LINE#         491
  C:0370H         LINE#         492
  C:0385H         LINE#         493
  C:0388H         LINE#         495
  C:0389H         LINE#         496
  C:0389H         LINE#         498
  C:0389H         LINE#         499
  C:0389H         LINE#         500
  C:038DH         LINE#         501
  C:038DH         LINE#         502
  C:038FH         LINE#         503
  C:0392H         LINE#         504
  C:0393H         LINE#         506
  C:0395H         LINE#         508
  C:0395H         LINE#         509
  C:0395H         LINE#         510
  C:0395H         LINE#         512
  C:0395H         LINE#         513
  C:0395H         LINE#         514
  C:0395H         LINE#         516
  C:0395H         LINE#         517
  -------         ENDPROC       TD_POLL
  -------         PROC          TD_SUSPEND
  C:0CFEH         LINE#         519
  C:0CFEH         LINE#         520
  C:0CFEH         LINE#         521
  C:0CFFH         LINE#         522
  -------         ENDPROC       TD_SUSPEND
  -------         PROC          TD_RESUME
  C:1078H         LINE#         524
  C:1078H         LINE#         525
BL51 BANKED LINKER/LOCATER V6.02                                                      04/19/2018  15:18:09  PAGE 40


  C:1078H         LINE#         526
  C:1079H         LINE#         527
  -------         ENDPROC       TD_RESUME
  -------         PROC          DR_GETDESCRIPTOR
  C:107AH         LINE#         534
  C:107AH         LINE#         535
  C:107AH         LINE#         536
  C:107BH         LINE#         537
  -------         ENDPROC       DR_GETDESCRIPTOR
  -------         PROC          DR_SETCONFIGURATION
  C:0AF8H         LINE#         539
  C:0AF8H         LINE#         540
  C:0AF8H         LINE#         541
  C:0AFEH         LINE#         542
  C:0AFFH         LINE#         543
  -------         ENDPROC       DR_SETCONFIGURATION
  -------         PROC          DR_GETCONFIGURATION
  C:101DH         LINE#         545
  C:101DH         LINE#         546
  C:101DH         LINE#         547
  C:1023H         LINE#         548
  C:1028H         LINE#         549
  C:102DH         LINE#         550
  C:102EH         LINE#         551
  -------         ENDPROC       DR_GETCONFIGURATION
  -------         PROC          DR_SETINTERFACE
  C:1064H         LINE#         553
  C:1064H         LINE#         554
  C:1064H         LINE#         555
  C:106AH         LINE#         556
  C:106BH         LINE#         557
  -------         ENDPROC       DR_SETINTERFACE
  -------         PROC          DR_GETINTERFACE
  C:102FH         LINE#         559
  C:102FH         LINE#         560
  C:102FH         LINE#         561
  C:1035H         LINE#         562
  C:103AH         LINE#         563
  C:103FH         LINE#         564
  C:1040H         LINE#         565
  -------         ENDPROC       DR_GETINTERFACE
  -------         PROC          DR_GETSTATUS
  C:107CH         LINE#         567
  C:107CH         LINE#         568
  C:107CH         LINE#         569
  C:107DH         LINE#         570
  -------         ENDPROC       DR_GETSTATUS
  -------         PROC          DR_CLEARFEATURE
  C:107EH         LINE#         572
  C:107EH         LINE#         573
  C:107EH         LINE#         574
  C:107FH         LINE#         575
  -------         ENDPROC       DR_CLEARFEATURE
  -------         PROC          DR_SETFEATURE
  C:1080H         LINE#         577
  C:1080H         LINE#         578
  C:1080H         LINE#         579
BL51 BANKED LINKER/LOCATER V6.02                                                      04/19/2018  15:18:09  PAGE 41


  C:1081H         LINE#         580
  -------         ENDPROC       DR_SETFEATURE
  -------         PROC          DR_VENDORCMND
  C:0396H         LINE#         584
  C:0396H         LINE#         585
  C:0396H         LINE#         586
  C:03E0H         LINE#         587
  C:03E0H         LINE#         631
  C:03E0H         LINE#         632
  C:03E0H         LINE#         633
  C:03E6H         LINE#         635
  C:03E6H         LINE#         636
  C:03E6H         LINE#         637
  C:03E6H         LINE#         638
  C:03E6H         LINE#         639
  C:03E9H         LINE#         640
  C:03E9H         LINE#         642
  C:03E9H         LINE#         643
  C:03E9H         LINE#         644
  C:03EFH         LINE#         646
  C:03EFH         LINE#         647
  C:03EFH         LINE#         648
  C:03EFH         LINE#         649
  C:03EFH         LINE#         650
  C:03F2H         LINE#         651
  C:03F2H         LINE#         653
  C:03F2H         LINE#         654
  C:03F2H         LINE#         655
  C:03F8H         LINE#         657
  C:03F8H         LINE#         658
  C:03F8H         LINE#         659
  C:03F8H         LINE#         660
  C:03F8H         LINE#         661
  C:03FBH         LINE#         662
  C:03FBH         LINE#         664
  C:03FBH         LINE#         665
  C:03FBH         LINE#         666
  C:0423H         LINE#         667
  C:0423H         LINE#         668
  C:0425H         LINE#         669
  C:042DH         LINE#         670
  C:0435H         LINE#         671
  C:043DH         LINE#         672
  C:0445H         LINE#         673
  C:044DH         LINE#         674
  C:0455H         LINE#         675
  C:045DH         LINE#         676
  C:0463H         LINE#         677
  C:0463H         LINE#         679
  C:0469H         LINE#         680
  C:046CH         LINE#         681
  C:046CH         LINE#         682
  C:046CH         LINE#         683
  C:046CH         LINE#         684
  C:046FH         LINE#         685
  C:046FH         LINE#         690
  C:046FH         LINE#         691
BL51 BANKED LINKER/LOCATER V6.02                                                      04/19/2018  15:18:09  PAGE 42


  C:046FH         LINE#         692
  C:0477H         LINE#         693
  C:0480H         LINE#         694
  C:0486H         LINE#         696
  C:0486H         LINE#         697
  C:0486H         LINE#         698
  C:0486H         LINE#         699
  C:0486H         LINE#         700
  C:0488H         LINE#         701
  C:0488H         LINE#         703
  C:0488H         LINE#         704
  C:0488H         LINE#         705
  C:0490H         LINE#         706
  C:0496H         LINE#         707
  C:049BH         LINE#         709
  C:049BH         LINE#         710
  C:049BH         LINE#         711
  C:049BH         LINE#         712
  C:049BH         LINE#         713
  C:049DH         LINE#         714
  C:049DH         LINE#         716
  C:049DH         LINE#         717
  C:049DH         LINE#         718
  C:04ABH         LINE#         719
  C:04B1H         LINE#         721
  C:04B6H         LINE#         722
  C:04B6H         LINE#         723
  C:04B6H         LINE#         724
  C:04B6H         LINE#         725
  C:04B8H         LINE#         726
  C:04B8H         LINE#         729
  C:04B8H         LINE#         730
  C:04B8H         LINE#         731
  C:04C7H         LINE#         732
  C:04CCH         LINE#         734
  C:04CFH         LINE#         736
  C:04D4H         LINE#         738
  C:04D4H         LINE#         739
  C:04D4H         LINE#         740
  C:04D4H         LINE#         741
  C:04D6H         LINE#         742
  C:04D6H         LINE#         744
  C:04D6H         LINE#         745
  C:04D6H         LINE#         746
  C:04E4H         LINE#         747
  C:04EAH         LINE#         749
  C:04EFH         LINE#         750
  C:04EFH         LINE#         751
  C:04EFH         LINE#         752
  C:04EFH         LINE#         753
  C:04F1H         LINE#         754
  C:04F1H         LINE#         756
  C:04F1H         LINE#         757
  C:04F1H         LINE#         758
  C:04F7H         LINE#         759
  C:04FBH         LINE#         760
  C:04FFH         LINE#         761
BL51 BANKED LINKER/LOCATER V6.02                                                      04/19/2018  15:18:09  PAGE 43


  C:0505H         LINE#         762
  C:0509H         LINE#         764
  C:050EH         LINE#         765
  C:0513H         LINE#         766
  C:0513H         LINE#         767
  C:0516H         LINE#         768
  C:0516H         LINE#         770
  C:0516H         LINE#         771
  C:0516H         LINE#         772
  C:051EH         LINE#         773
  C:0523H         LINE#         774
  C:0527H         LINE#         775
  C:0527H         LINE#         776
  C:052AH         LINE#         777
  C:052AH         LINE#         779
  C:052AH         LINE#         780
  C:052AH         LINE#         781
  C:0532H         LINE#         782
  C:0537H         LINE#         783
  C:053BH         LINE#         784
  C:053BH         LINE#         785
  C:053EH         LINE#         786
  C:053EH         LINE#         788
  C:053EH         LINE#         789
  C:053EH         LINE#         790
  C:0546H         LINE#         791
  C:054BH         LINE#         792
  C:054FH         LINE#         793
  C:054FH         LINE#         794
  C:0552H         LINE#         795
  C:0552H         LINE#         797
  C:0552H         LINE#         798
  C:0552H         LINE#         799
  C:055AH         LINE#         800
  C:055FH         LINE#         801
  C:0563H         LINE#         802
  C:0563H         LINE#         803
  C:0566H         LINE#         804
  C:0566H         LINE#         806
  C:0566H         LINE#         807
  C:0566H         LINE#         808
  C:056EH         LINE#         809
  C:0576H         LINE#         810
  C:057BH         LINE#         811
  C:057FH         LINE#         812
  C:057FH         LINE#         813
  C:0582H         LINE#         814
  C:0582H         LINE#         816
  C:0582H         LINE#         817
  C:0582H         LINE#         818
  C:058AH         LINE#         819
  C:0592H         LINE#         820
  C:0597H         LINE#         821
  C:059BH         LINE#         822
  C:059BH         LINE#         823
  C:059EH         LINE#         824
  C:059EH         LINE#         826
BL51 BANKED LINKER/LOCATER V6.02                                                      04/19/2018  15:18:09  PAGE 44


  C:059EH         LINE#         827
  C:059EH         LINE#         828
  C:05A6H         LINE#         829
  C:05AEH         LINE#         830
  C:05B3H         LINE#         831
  C:05B7H         LINE#         832
  C:05B7H         LINE#         833
  C:05BAH         LINE#         834
  C:05BAH         LINE#         836
  C:05BAH         LINE#         837
  C:05BAH         LINE#         838
  C:05C2H         LINE#         839
  C:05CAH         LINE#         840
  C:05CFH         LINE#         841
  C:05D3H         LINE#         842
  C:05D3H         LINE#         843
  C:05D6H         LINE#         844
  C:05D6H         LINE#         908
  C:05D6H         LINE#         909
  C:05D6H         LINE#         910
  C:05DCH         LINE#         911
  C:05E1H         LINE#         912
  C:05E6H         LINE#         913
  C:05EBH         LINE#         914
  C:05F2H         LINE#         916
  C:05FBH         LINE#         917
  C:05FBH         LINE#         918
  C:05FBH         LINE#         919
  C:05FBH         LINE#         920
  C:05FDH         LINE#         921
  C:05FFH         LINE#         922
  C:0601H         LINE#         923
  C:0601H         LINE#         925
  C:0601H         LINE#         926
  C:0601H         LINE#         927
  C:0604H         LINE#         928
  C:0606H         LINE#         929
  C:0608H         LINE#         930
  C:060AH         LINE#         931
  C:060AH         LINE#         932
  C:060AH         LINE#         934
  C:060AH         LINE#         935
  C:060AH         LINE#         937
  C:060AH         LINE#         938
  C:060AH         LINE#         939
  C:0613H         LINE#         940
  C:0613H         LINE#         941
  C:0613H         LINE#         942
  C:0613H         LINE#         943
  C:061BH         LINE#         944
  C:0621H         LINE#         945
  C:0623H         LINE#         946
  C:0623H         LINE#         948
  C:0623H         LINE#         949
  C:0623H         LINE#         950
  C:062BH         LINE#         951
  C:0631H         LINE#         952
BL51 BANKED LINKER/LOCATER V6.02                                                      04/19/2018  15:18:09  PAGE 45


  C:0631H         LINE#         953
  C:0631H         LINE#         954
  C:0631H         LINE#         956
  C:0639H         LINE#         957
  C:0641H         LINE#         958
  C:0646H         LINE#         959
  C:064BH         LINE#         960
  C:064BH         LINE#         962
  C:064DH         LINE#         963
  C:064DH         LINE#         965
  C:064DH         LINE#         966
  C:064DH         LINE#         967
  C:065EH         LINE#         968
  C:0663H         LINE#         969
  C:0668H         LINE#         970
  C:066FH         LINE#         972
  C:0671H         LINE#         973
  C:0671H         LINE#         975
  C:0671H         LINE#         976
  C:0673H         LINE#         977
  C:0673H         LINE#         978
  C:0674H         LINE#         979
  -------         ENDPROC       DR_VENDORCMND
  -------         PROC          ISR_SUDAV
  C:0F92H         LINE#         987
  C:0F98H         LINE#         991
  C:0F9FH         LINE#         992
  C:0FA1H         LINE#         993
  C:0FA4H         LINE#         994
  C:0FAAH         LINE#         995
  -------         ENDPROC       ISR_SUDAV
  -------         PROC          ISR_SUTOK
  C:0FC9H         LINE#         998
  C:0FCFH         LINE#         1000
  C:0FD2H         LINE#         1001
  C:0FD8H         LINE#         1002
  -------         ENDPROC       ISR_SUTOK
  -------         PROC          ISR_SOF
  C:0FDFH         LINE#         1004
  C:0FE5H         LINE#         1006
  C:0FE8H         LINE#         1007
  C:0FEEH         LINE#         1008
  -------         ENDPROC       ISR_SOF
  -------         PROC          ISR_URES
  C:0C96H         LINE#         1010
  C:0C9CH         LINE#         1012
  C:0CA3H         LINE#         1013
  C:0CA3H         LINE#         1014
  C:0CA9H         LINE#         1015
  C:0CAFH         LINE#         1016
  C:0CB5H         LINE#         1018
  C:0CB7H         LINE#         1020
  C:0CB7H         LINE#         1021
  C:0CBDH         LINE#         1022
  C:0CC3H         LINE#         1023
  C:0CC9H         LINE#         1024
  C:0CC9H         LINE#         1026
BL51 BANKED LINKER/LOCATER V6.02                                                      04/19/2018  15:18:09  PAGE 46


  C:0CCCH         LINE#         1027
  C:0CD2H         LINE#         1028
  -------         ENDPROC       ISR_URES
  -------         PROC          ISR_SUSP
  C:0FB1H         LINE#         1030
  C:0FB7H         LINE#         1032
  C:0FB9H         LINE#         1033
  C:0FBCH         LINE#         1034
  C:0FC2H         LINE#         1035
  -------         ENDPROC       ISR_SUSP
  -------         PROC          ISR_HIGHSPEED
  C:0D72H         LINE#         1037
  C:0D78H         LINE#         1039
  C:0D7FH         LINE#         1040
  C:0D7FH         LINE#         1041
  C:0D85H         LINE#         1042
  C:0D8BH         LINE#         1043
  C:0D91H         LINE#         1045
  C:0D93H         LINE#         1047
  C:0D93H         LINE#         1048
  C:0D99H         LINE#         1049
  C:0D9FH         LINE#         1050
  C:0DA5H         LINE#         1051
  C:0DA5H         LINE#         1053
  C:0DA8H         LINE#         1054
  C:0DAEH         LINE#         1055
  -------         ENDPROC       ISR_HIGHSPEED
  -------         PROC          TIMER0_INIT
  C:0F50H         LINE#         1059
  C:0F50H         LINE#         1060
  C:0F50H         LINE#         1061
  C:0F52H         LINE#         1062
  C:0F57H         LINE#         1063
  C:0F59H         LINE#         1064
  C:0F5CH         LINE#         1065
  C:0F5FH         LINE#         1066
  C:0F62H         LINE#         1067
  C:0F65H         LINE#         1068
  C:0F68H         LINE#         1069
  C:0F6AH         LINE#         1070
  C:0F6CH         LINE#         1071
  C:0F6EH         LINE#         1072
  C:0F70H         LINE#         1073
  -------         ENDPROC       TIMER0_INIT
  -------         PROC          TIMER1_INIT
  C:0F71H         LINE#         1077
  C:0F71H         LINE#         1078
  C:0F71H         LINE#         1079
  C:0F73H         LINE#         1080
  C:0F78H         LINE#         1081
  C:0F7AH         LINE#         1082
  C:0F7DH         LINE#         1083
  C:0F80H         LINE#         1084
  C:0F83H         LINE#         1085
  C:0F86H         LINE#         1086
  C:0F89H         LINE#         1087
  C:0F8BH         LINE#         1088
BL51 BANKED LINKER/LOCATER V6.02                                                      04/19/2018  15:18:09  PAGE 47


  C:0F8DH         LINE#         1090
  C:0F8FH         LINE#         1091
  C:0F91H         LINE#         1092
  -------         ENDPROC       TIMER1_INIT
  -------         PROC          INICIALIZARPUERTOS
  C:0EE8H         LINE#         1094
  C:0EE8H         LINE#         1095
  C:0EE8H         LINE#         1115
  C:0EEBH         LINE#         1119
  C:0EEDH         LINE#         1120
  C:0EEFH         LINE#         1121
  C:0EF1H         LINE#         1122
  C:0EF3H         LINE#         1123
  C:0EF5H         LINE#         1124
  C:0EF7H         LINE#         1125
  C:0EF9H         LINE#         1129
  C:0EFCH         LINE#         1130
  C:0EFEH         LINE#         1131
  C:0F00H         LINE#         1132
  C:0F02H         LINE#         1134
  C:0F04H         LINE#         1135
  C:0F06H         LINE#         1136
  C:0F08H         LINE#         1137
  C:0F0AH         LINE#         1138
  C:0F0CH         LINE#         1140
  -------         ENDPROC       INICIALIZARPUERTOS
  -------         PROC          _ANTIREBOTEPEDALES
  D:0007H         SYMBOL        pedal
  -------         DO            
  B:0020H.5       SYMBOL        ret
  -------         ENDDO         
  C:0A13H         LINE#         1142
  C:0A13H         LINE#         1143
  C:0A13H         LINE#         1146
  C:0A28H         LINE#         1147
  C:0A28H         LINE#         1148
  C:0A28H         LINE#         1149
  C:0A28H         LINE#         1150
  C:0A33H         LINE#         1151
  C:0A33H         LINE#         1152
  C:0A33H         LINE#         1153
  C:0A33H         LINE#         1154
  C:0A37H         LINE#         1155
  C:0A39H         LINE#         1156
  C:0A39H         LINE#         1158
  C:0A39H         LINE#         1159
  C:0A39H         LINE#         1160
  C:0A3DH         LINE#         1161
  C:0A3FH         LINE#         1162
  C:0A3FH         LINE#         1164
  C:0A3FH         LINE#         1165
  C:0A3FH         LINE#         1166
  C:0A43H         LINE#         1167
  C:0A43H         LINE#         1168
  C:0A43H         LINE#         1169
  C:0A43H         LINE#         1171
  C:0A46H         LINE#         1172
BL51 BANKED LINKER/LOCATER V6.02                                                      04/19/2018  15:18:09  PAGE 48


  C:0A48H         LINE#         1173
  C:0A49H         LINE#         1174
  C:0A49H         LINE#         1176
  C:0A49H         LINE#         1177
  C:0A49H         LINE#         1178
  C:0A54H         LINE#         1179
  C:0A54H         LINE#         1180
  C:0A54H         LINE#         1181
  C:0A54H         LINE#         1182
  C:0A58H         LINE#         1183
  C:0A5AH         LINE#         1184
  C:0A5AH         LINE#         1186
  C:0A5AH         LINE#         1187
  C:0A5AH         LINE#         1188
  C:0A5EH         LINE#         1189
  C:0A60H         LINE#         1190
  C:0A60H         LINE#         1192
  C:0A60H         LINE#         1193
  C:0A60H         LINE#         1194
  C:0A64H         LINE#         1195
  C:0A64H         LINE#         1196
  C:0A64H         LINE#         1197
  C:0A64H         LINE#         1199
  C:0A67H         LINE#         1200
  C:0A6AH         LINE#         1202
  C:0A6CH         LINE#         1204
  C:0A6DH         LINE#         1205
  C:0A6DH         LINE#         1207
  C:0A6DH         LINE#         1208
  C:0A6DH         LINE#         1209
  C:0A78H         LINE#         1210
  C:0A78H         LINE#         1211
  C:0A78H         LINE#         1212
  C:0A78H         LINE#         1213
  C:0A7CH         LINE#         1214
  C:0A7EH         LINE#         1215
  C:0A7EH         LINE#         1217
  C:0A7EH         LINE#         1218
  C:0A7EH         LINE#         1219
  C:0A82H         LINE#         1220
  C:0A84H         LINE#         1221
  C:0A84H         LINE#         1223
  C:0A84H         LINE#         1224
  C:0A84H         LINE#         1225
  C:0A88H         LINE#         1226
  C:0A88H         LINE#         1227
  C:0A88H         LINE#         1228
  C:0A88H         LINE#         1230
  C:0A8BH         LINE#         1231
  C:0A8EH         LINE#         1233
  C:0A90H         LINE#         1235
  C:0A91H         LINE#         1236
  C:0A91H         LINE#         1238
  C:0A91H         LINE#         1239
  C:0A91H         LINE#         1240
  C:0A9CH         LINE#         1241
  C:0A9CH         LINE#         1242
BL51 BANKED LINKER/LOCATER V6.02                                                      04/19/2018  15:18:09  PAGE 49


  C:0A9CH         LINE#         1243
  C:0A9CH         LINE#         1244
  C:0AA0H         LINE#         1245
  C:0AA2H         LINE#         1246
  C:0AA2H         LINE#         1248
  C:0AA2H         LINE#         1249
  C:0AA2H         LINE#         1250
  C:0AA6H         LINE#         1251
  C:0AA8H         LINE#         1252
  C:0AA8H         LINE#         1254
  C:0AA8H         LINE#         1255
  C:0AA8H         LINE#         1256
  C:0AACH         LINE#         1257
  C:0AACH         LINE#         1258
  C:0AACH         LINE#         1259
  C:0AACH         LINE#         1261
  C:0AAFH         LINE#         1262
  C:0AB1H         LINE#         1264
  C:0AB1H         LINE#         1265
  C:0AB1H         LINE#         1266
  C:0AB1H         LINE#         1267
  -------         ENDPROC       _ANTIREBOTEPEDALES
  -------         PROC          ISR_EP0ACK
  C:1082H         LINE#         1270
  C:1082H         LINE#         1272
  -------         ENDPROC       ISR_EP0ACK
  -------         PROC          ISR_STUB
  C:1083H         LINE#         1273
  C:1083H         LINE#         1275
  -------         ENDPROC       ISR_STUB
  -------         PROC          ISR_EP0IN
  C:1084H         LINE#         1276
  C:1084H         LINE#         1278
  -------         ENDPROC       ISR_EP0IN
  -------         PROC          ISR_EP0OUT
  C:1085H         LINE#         1279
  C:1085H         LINE#         1281
  -------         ENDPROC       ISR_EP0OUT
  -------         PROC          ISR_EP1IN
  C:1086H         LINE#         1282
  C:1086H         LINE#         1284
  -------         ENDPROC       ISR_EP1IN
  -------         PROC          ISR_EP1OUT
  C:1087H         LINE#         1285
  C:1087H         LINE#         1287
  -------         ENDPROC       ISR_EP1OUT
  -------         PROC          ISR_EP2INOUT
  C:1088H         LINE#         1288
  C:1088H         LINE#         1290
  -------         ENDPROC       ISR_EP2INOUT
  -------         PROC          ISR_EP4INOUT
  C:1089H         LINE#         1291
  C:1089H         LINE#         1293
  -------         ENDPROC       ISR_EP4INOUT
  -------         PROC          ISR_EP6INOUT
  C:108AH         LINE#         1294
  C:108AH         LINE#         1296
BL51 BANKED LINKER/LOCATER V6.02                                                      04/19/2018  15:18:09  PAGE 50


  -------         ENDPROC       ISR_EP6INOUT
  -------         PROC          ISR_EP8INOUT
  C:108BH         LINE#         1297
  C:108BH         LINE#         1299
  -------         ENDPROC       ISR_EP8INOUT
  -------         PROC          ISR_IBN
  C:108CH         LINE#         1300
  C:108CH         LINE#         1302
  -------         ENDPROC       ISR_IBN
  -------         PROC          ISR_EP0PINGNAK
  C:108DH         LINE#         1303
  C:108DH         LINE#         1305
  -------         ENDPROC       ISR_EP0PINGNAK
  -------         PROC          ISR_EP1PINGNAK
  C:108EH         LINE#         1306
  C:108EH         LINE#         1308
  -------         ENDPROC       ISR_EP1PINGNAK
  -------         PROC          ISR_EP2PINGNAK
  C:108FH         LINE#         1309
  C:108FH         LINE#         1311
  -------         ENDPROC       ISR_EP2PINGNAK
  -------         PROC          ISR_EP4PINGNAK
  C:1090H         LINE#         1312
  C:1090H         LINE#         1314
  -------         ENDPROC       ISR_EP4PINGNAK
  -------         PROC          ISR_EP6PINGNAK
  C:1091H         LINE#         1315
  C:1091H         LINE#         1317
  -------         ENDPROC       ISR_EP6PINGNAK
  -------         PROC          ISR_EP8PINGNAK
  C:1092H         LINE#         1318
  C:1092H         LINE#         1320
  -------         ENDPROC       ISR_EP8PINGNAK
  -------         PROC          ISR_ERRORLIMIT
  C:1093H         LINE#         1321
  C:1093H         LINE#         1323
  -------         ENDPROC       ISR_ERRORLIMIT
  -------         PROC          ISR_EP2PIDERROR
  C:1094H         LINE#         1324
  C:1094H         LINE#         1326
  -------         ENDPROC       ISR_EP2PIDERROR
  -------         PROC          ISR_EP4PIDERROR
  C:1095H         LINE#         1327
  C:1095H         LINE#         1329
  -------         ENDPROC       ISR_EP4PIDERROR
  -------         PROC          ISR_EP6PIDERROR
  C:1096H         LINE#         1330
  C:1096H         LINE#         1332
  -------         ENDPROC       ISR_EP6PIDERROR
  -------         PROC          ISR_EP8PIDERROR
  C:1097H         LINE#         1333
  C:1097H         LINE#         1335
  -------         ENDPROC       ISR_EP8PIDERROR
  -------         PROC          ISR_EP2PFLAG
  C:1098H         LINE#         1336
  C:1098H         LINE#         1338
  -------         ENDPROC       ISR_EP2PFLAG
BL51 BANKED LINKER/LOCATER V6.02                                                      04/19/2018  15:18:09  PAGE 51


  -------         PROC          ISR_EP4PFLAG
  C:1099H         LINE#         1339
  C:1099H         LINE#         1341
  -------         ENDPROC       ISR_EP4PFLAG
  -------         PROC          ISR_EP6PFLAG
  C:109AH         LINE#         1342
  C:109AH         LINE#         1344
  -------         ENDPROC       ISR_EP6PFLAG
  -------         PROC          ISR_EP8PFLAG
  C:109BH         LINE#         1345
  C:109BH         LINE#         1347
  -------         ENDPROC       ISR_EP8PFLAG
  -------         PROC          ISR_EP2EFLAG
  C:109CH         LINE#         1348
  C:109CH         LINE#         1350
  -------         ENDPROC       ISR_EP2EFLAG
  -------         PROC          ISR_EP4EFLAG
  C:109DH         LINE#         1351
  C:109DH         LINE#         1353
  -------         ENDPROC       ISR_EP4EFLAG
  -------         PROC          ISR_EP6EFLAG
  C:109EH         LINE#         1354
  C:109EH         LINE#         1356
  -------         ENDPROC       ISR_EP6EFLAG
  -------         PROC          ISR_EP8EFLAG
  C:109FH         LINE#         1357
  C:109FH         LINE#         1359
  -------         ENDPROC       ISR_EP8EFLAG
  -------         PROC          ISR_EP2FFLAG
  C:10A0H         LINE#         1360
  C:10A0H         LINE#         1362
  -------         ENDPROC       ISR_EP2FFLAG
  -------         PROC          ISR_EP4FFLAG
  C:10A1H         LINE#         1363
  C:10A1H         LINE#         1365
  -------         ENDPROC       ISR_EP4FFLAG
  -------         PROC          ISR_EP6FFLAG
  C:10A2H         LINE#         1366
  C:10A2H         LINE#         1368
  -------         ENDPROC       ISR_EP6FFLAG
  -------         PROC          ISR_EP8FFLAG
  C:10A3H         LINE#         1369
  C:10A3H         LINE#         1371
  -------         ENDPROC       ISR_EP8FFLAG
  -------         PROC          ISR_GPIFCOMPLETE
  C:10A4H         LINE#         1372
  C:10A4H         LINE#         1374
  -------         ENDPROC       ISR_GPIFCOMPLETE
  -------         PROC          ISR_GPIFWAVEFORM
  C:10A5H         LINE#         1375
  C:10A5H         LINE#         1377
  -------         ENDPROC       ISR_GPIFWAVEFORM
  -------         ENDMOD        PEDALERA

  -------         MODULE        I2C
  C:0000H         SYMBOL        _ICE_DUMMY_
  C:0FF5H         PUBLIC        I2CWaitForAck
BL51 BANKED LINKER/LOCATER V6.02                                                      04/19/2018  15:18:09  PAGE 52


  C:106CH         PUBLIC        I2CWaitForStop
  C:1041H         PUBLIC        _I2CStartAndAddrW
  C:0F0DH         PUBLIC        _SetDAC5571
  C:0C44H         PUBLIC        _I2CWrite
  -------         PROC          _I2CWRITE
  D:0018H         SYMBOL        addr
  D:0019H         SYMBOL        length
  D:001AH         SYMBOL        buf
  -------         DO            
  D:001CH         SYMBOL        i
  -------         ENDDO         
  C:0C44H         LINE#         39
  C:0C4CH         LINE#         40
  C:0C4CH         LINE#         42
  C:0C4FH         LINE#         43
  C:0C52H         LINE#         44
  C:0C57H         LINE#         45
  C:0C58H         LINE#         46
  C:0C5EH         LINE#         47
  C:0C63H         LINE#         48
  C:0C64H         LINE#         50
  C:0C6EH         LINE#         51
  C:0C6EH         LINE#         52
  C:0C7EH         LINE#         53
  C:0C83H         LINE#         54
  C:0C84H         LINE#         55
  C:0C88H         LINE#         57
  C:0C8EH         LINE#         58
  C:0C94H         LINE#         59
  C:0C95H         LINE#         60
  -------         ENDPROC       _I2CWRITE
  -------         PROC          I2CWAITFORSTOP
  C:106CH         LINE#         62
  C:106CH         LINE#         63
  C:106CH         LINE#         65
  C:1073H         LINE#         66
  -------         ENDPROC       I2CWAITFORSTOP
  -------         PROC          I2CWAITFORACK
  -------         DO            
  D:0007H         SYMBOL        i
  -------         ENDDO         
  C:0FF5H         LINE#         97
  C:0FF5H         LINE#         98
  C:0FF5H         LINE#         101
  C:0FFDH         LINE#         103
  C:1001H         LINE#         104
  C:1003H         LINE#         105
  C:1007H         LINE#         106
  C:1009H         LINE#         108
  C:100AH         LINE#         109
  -------         ENDPROC       I2CWAITFORACK
  -------         PROC          _I2CSTARTANDADDRW
  D:0007H         SYMBOL        address_w
  C:1041H         LINE#         111
  C:1041H         LINE#         112
  C:1041H         LINE#         113
  C:1047H         LINE#         114
BL51 BANKED LINKER/LOCATER V6.02                                                      04/19/2018  15:18:09  PAGE 53


  C:104EH         LINE#         115
  -------         ENDPROC       _I2CSTARTANDADDRW
  -------         PROC          _SETDAC5571
  D:0004H         SYMBOL        valor
  D:0005H         SYMBOL        modo
  -------         DO            
  X:2000H         SYMBOL        buff
  -------         ENDDO         
  C:0F0DH         LINE#         126
  C:0F0FH         LINE#         127
  C:0F0FH         LINE#         129
  C:0F1DH         LINE#         130
  C:0F23H         LINE#         131
  C:0F2EH         LINE#         132
  -------         ENDPROC       _SETDAC5571
  -------         ENDMOD        I2C

  -------         MODULE        ?C?ULCMP
  C:0E2BH         PUBLIC        ?C?ULCMP
  -------         ENDMOD        ?C?ULCMP

  -------         MODULE        ?C?CCASE
  C:0E3CH         PUBLIC        ?C?CCASE
  -------         ENDMOD        ?C?CCASE

Program Size: data=74.6 xdata=4475 code=4152
LINK/LOCATE RUN COMPLETE.  0 WARNING(S),  0 ERROR(S)
